:020000040000FA
:10000000605B01203D02000061020000630200000D
:100010006502000067020000690200006B02000038
:100020006B0200006B0200006B0200006B0200001C
:100030006B0200006B020000270300000524000093
:10004000910600009B060000A5060000AF06000018
:10005000B9060000B1090000BB090000D508000086
:10006000DB07000049080000530800005D0800009D
:10007000670800007B080000ED050000F7050000A0
:10008000010600000B0600001F0A00001109000015
:100090001B090000250900002F0900003909000094
:1000A00043090000CF050000D9050000E30500006A
:1000B000FD0800007D060000C3060000CD0600001C
:1000C000D7060000C5090000DF0800004D09000048
:1000D00057090000E5070000470600005106000030
:1000E00073060000D1070000150A00007108000027
:1000F0000B0A0000010A0000150600001F060000A0
:10010000290600003306000069060000E106000031
:10011000EB060000F5060000E9080000F308000007
:10012000CF090000D9090000E3090000ED09000033
:10013000F7090000EF070000F9070000610900005F
:100140006B090000750900007F09000087060000A8
:10015000AD080000B7080000030800000D0800000B
:10016000FF06000009070000C108000007090000A1
:10017000130700001D0700002707000031070000DB
:100180003B070000450700004F070000590700002B
:10019000630700006D07000077070000810700007B
:1001A0008B070000950700009F070000A9070000CB
:1001B000B3070000BD070000CB0800003D060000AB
:1001C0005B0600003F080000890900009309000059
:1001D0009D090000A7090000170800002108000081
:1001E00085080000C50500008F0800009908000080
:1001F000A30800002B08000035080000C707000016
:10020000DFF80CD000F024F90048004725850000F5
:10021000605B0120EFF3108072B67047EFF310803F
:100220007047EFF3108062B6704730BF704780F3BD
:1002300011887047EFF3118070470000DFF830003D
:10024000016841F470010160BFF34F8FDFF82400B3
:10025000016821F040410160BFF36F8F06480047FD
:10026000FEE7FEE7FEE7FEE7FEE7FEE7FEE700004B
:1002700088ED00E034EF00E00102000072B6704744
:1002800062B67047EFF3108072B6704780F3108843
:10029000704730BF704720BF7047B0FA80F070479A
:1002A00090FAA0F0B0FA80F0704790FAA0F0704792
:1002B000EFF3098141B1F1EE101A40F8041D20ED71
:1002C000200A29490A6810607047B0EC200A02C869
:1002D000E1EE101A25490A6810607047EFF31080AC
:1002E00072B6704780F31088704721484FF0FF01C5
:1002F0000170002080F309881E48016881F3088896
:100300001D48012101701D484FF08051016062B607
:10031000FEE71A484FF080510160704717484FF0D0
:1003200080510160704772B6EFF3098028B1203820
:1003300080E8F00F0C490968086000B51048804754
:100340005DF804EB0F4810490A7802700648074927
:100350000A680260106890E8F00F203080F3098886
:100360004EF0F40E62B670473800002040000020C6
:1003700022ED00E0700000203200002004ED00E0DB
:100380008D1F000027000020280000200048704733
:10039000E896000040EA01039B0703D009E008C982
:1003A000121F08C0042AFAD203E011F8013B00F83A
:1003B000013B521EF9D27047D2B201E000F8012B86
:1003C000491EFBD270470022F6E710B513460A46D5
:1003D00004461946FFF7F0FF204610BD30B505462C
:1003E0002A460B4612F8010B13F8014B08B1A04244
:1003F000F8D01CB1002802D06D1CF1E7284630BDB2
:10040000CAB2401E10F8011F8A4202D00029F9D159
:1004100000207047421C10F8011B0029FBD1801AF4
:10042000704730B50B46014600202022012409E028
:1004300021FA02F59D4205D303FA02F5491B04FA9D
:1004400002F52844151EA2F10102F1DC30BD0000C6
:10045000064C074D06E0E06840F0010394E8070011
:1004600098471034AC42F6D3FFF7CEFEEC9600006E
:100470000C97000070B58C1810F8015B15F007039D
:1004800001D110F8013B2A1106D110F8012B03E02D
:1004900010F8016B01F8016B5B1EF9D12B0705D435
:1004A0000023521E0DD401F8013BFAE710F8013B7E
:1004B000CB1A921C03E013F8015B01F8015B521E9A
:1004C000F9D5A142D8D3002070BD000038B504F0A2
:1004D00073FC05F09DFC05F075FC02F0A1FC02F038
:1004E00087FC02F063FC00BF6A46192103A000F0FC
:1004F000A3FC0446002CF7D038BD000041707054B6
:1005000061736B4372656174653A204A6F696E204E
:10051000696E21210A00000000F023F800F0ACFA17
:1005200004464FF47A70B4FBF0F5284601F07EFFE4
:1005300000F05CFB01F0F4F900F0E4FEFFF7C6FF09
:1005400006E04FF4FA7300221146104601F05EFDFA
:10055000F7E77047704770477047704770477047BC
:10056000704710B500F060FA00F0E0FA10BD10B569
:100570000446702C04D204F11001C8B200F03CFB18
:1005800010BD000070B50446002600BF00BFFFF795
:1005900079FE064600BF00BF01F01EF800BF00BF95
:1005A0003046FFF773FE00BF00BF702C04D2044832
:1005B00050F8245005B1A84701F028F870BD00009C
:1005C000B005002010B56920FFF7DCFF10BD10B5A5
:1005D0001920FFF7D7FF10BD10B51A20FFF7D2FF83
:1005E00010BD10B51B20FFF7CDFF10BD10B50E20BC
:1005F000FFF7C8FF10BD10B50F20FFF7C3FF10BDF8
:1006000010B51020FFF7BEFF10BD10B51120FFF789
:10061000B9FF10BD10B52E20FFF7B4FF10BD10B507
:100620002F20FFF7AFFF10BD10B53020FFF7AAFF56
:1006300010BD10B53120FFF7A5FF10BD10B55F202C
:10064000FFF7A0FF10BD10B52620FFF79BFF10BDE0
:1006500010B52720FFF796FF10BD10B56020FFF7FB
:1006600091FF10BD00BFFEE710B53220FFF78AFFF3
:1006700010BD10B52820FFF785FF10BD10B51D2057
:10068000FFF780FF10BD10B54320FFF77BFF10BDC3
:1006900010B50020FFF776FF10BD10B50120FFF761
:1006A00071FF10BD10B50220FFF76CFF10BD10B533
:1006B0000320FFF767FF10BD10B50420FFF762FFAE
:1006C00010BD10B51E20FFF75DFF10BD10B51F2037
:1006D000FFF758FF10BD10B52020FFF753FF10BDE6
:1006E00010B53320FFF74EFF10BD10B53420FFF7D3
:1006F00049FF10BD10B53520FFF744FF10BD10B500
:100700004820FFF73FFF10BD10B54920FFF73AFF23
:1007100010BD10B54C20FFF735FF10BD10B54D20B2
:10072000FFF730FF10BD10B54E20FFF72BFF10BDB7
:1007300010B54F20FFF726FF10BD10B55020FFF772
:1007400021FF10BD10B55120FFF71CFF10BD10B5E3
:100750005220FFF717FF10BD10B55320FFF712FF0F
:1007600010BD10B55420FFF70DFF10BD10B555207A
:10077000FFF708FF10BD10B55620FFF703FF10BDAF
:1007800010B55720FFF7FEFE10BD10B55820FFF73B
:10079000F9FE10BD10B55920FFF7F4FE10BD10B5DD
:1007A0005A20FFF7EFFE10BD10B55B20FFF7EAFE01
:1007B00010BD10B55C20FFF7E5FE10BD10B55D2043
:1007C000FFF7E0FE10BD10B56F20FFF7DBFE10BD98
:1007D00010B52920FFF7D6FE10BD10B50820FFF791
:1007E000D1FE10BD10B52520FFF7CCFE10BD10B511
:1007F0003D20FFF7C7FE10BD10B53E20FFF7C2FE3B
:1008000010BD10B54620FFF7BDFE10BD10B5472046
:10081000FFF7B8FE10BD10B56620FFF7B3FE10BDA0
:1008200010B56720FFF7AEFE10BD10B56D20FFF7C5
:10083000A9FE10BD10B56E20FFF7A4FE10BD10B5C7
:100840006120FFF79FFE10BD10B50920FFF79AFE4B
:1008500010BD10B50A20FFF795FE10BD10B50B2096
:10086000FFF790FE10BD10B50C20FFF78BFE10BDFA
:1008700010B52B20FFF786FE10BD10B50D20FFF739
:1008800081FE10BD10B56820FFF77CFE10BD10B5CD
:100890006A20FFF777FE10BD10B56B20FFF772FEE0
:1008A00010BD10B56C20FFF76DFE10BD10B54420D3
:1008B000FFF768FE10BD10B54520FFF763FE10BDC1
:1008C00010B54A20FFF75EFE10BD10B55E20FFF7A1
:1008D00059FE10BD10B50720FFF754FE10BD10B52E
:1008E0002220FFF74FFE10BD10B53620FFF74AFE5D
:1008F00010BD10B53720FFF745FE10BD10B51C2008
:10090000FFF740FE10BD10B54B20FFF73BFE10BDBA
:1009100010B51320FFF736FE10BD10B51420FFF7F9
:1009200031FE10BD10B51520FFF72CFE10BD10B51F
:100930001620FFF727FE10BD10B51720FFF722FE87
:1009400010BD10B51820FFF71DFE10BD10B52320F7
:10095000FFF718FE10BD10B52420FFF713FE10BDE1
:1009600010B53F20FFF70EFE10BD10B54020FFF779
:1009700009FE10BD10B54120FFF704FE10BD10B5F3
:100980004220FFF7FFFD10BD10B56220FFF7FAFD12
:1009900010BD10B56320FFF7F5FD10BD10B5642044
:1009A000FFF7F0FD10BD10B56520FFF7EBFD10BDA2
:1009B00010B50520FFF7E6FD10BD10B50620FFF7C6
:1009C000E1FD10BD10B52120FFF7DCFD10BD10B515
:1009D0003820FFF7D7FD10BD10B53920FFF7D2FD45
:1009E00010BD10B53A20FFF7CDFD10BD10B53B206E
:1009F000FFF7C8FD10BD10B53C20FFF7C3FD10BDCB
:100A000010B52D20FFF7BEFD10BD10B52C20FFF74F
:100A1000B9FD10BD10B52A20FFF7B4FD10BD10B50B
:100A20001220FFF7AFFD10BD10B5002404E0E0B2C6
:100A3000034900F007F8641C702CF8D310BD0000C7
:100A40006506000070B504460D460026702C10D2D5
:100A500000BF00BFFFF716FC064600BF00BF0548F9
:100A600040F8245000BF00BF3046FFF70FFC00BF26
:100A700000BF70BDB00500202DE9F043DFF89CC039
:100A8000DCF8B0C0CCF3007CBCF1000F3ED0DFF846
:100A90008CC0DCF860C1CCF38A26DFF880C0DCF8BB
:100AA00060C1CCF30A0303EB9622DFF870C0DCF8D8
:100AB00064C1CCF30424DFF864C0DCF864C10CF03A
:100AC0001F05DFF858C0DCF8B0C0CCF3036111B1EA
:100AD000032904D101E0124902E0124900E000BFFD
:100AE00000BF01FB02F804F1010C05F101090CFB48
:100AF00009FCB8FBFCF0DFF824C0DCF8B0C0CCF394
:100B0000090C0CF10107B0FBF7F000E00020DFF862
:100B100018C0CCF80000BDE8F083000000E00F40F2
:100B20000024F40040787D01080000202948C06FAF
:100B300020F01C002749C8670846C06F40F010002D
:100B4000C8672448C0300068234908402149C1F8DB
:100B5000C0002048C0300068204908431D49C0310A
:100B6000086048061B49B03108604FF04C700860BF
:100B700060201B49086004201649C1F86401184828
:100B8000A0380068144908401249C1F8C000144850
:100B9000A0380068134908430E49C1F8C000084650
:100BA000D0F8600140F40000C1F8600100BF0C48BB
:100BB0000830006800F0010080F001000028F6D144
:100BC0000448B0300068084908430249C1F8B00041
:100BD0007047000000E00F4010FC10FC8100010095
:100BE00060E10F40850185010300009010B500F021
:100BF000F9F800F0BFF810BD2DE9F04104464FF0C0
:100C00000008102C6BD2DFE804F0080E0F10142936
:100C10003E090A0B0C11120D135300BF00BF00BF99
:100C200000BF00BF89E000BF00BF00BF00BF00BF22
:100C300083E000BF00BFFFF725FB804600BF00BF79
:100C40003F48006840F480303D49086000BF00BF65
:100C50004046FFF71BFB00BF00BF6EE000BF00BFB8
:100C6000FFF710FB804600BF00BF3548006840F426
:100C700000303349086000BF00BF4046FFF706FB65
:100C800000BF00BF59E000BF00BFFFF7FBFA80467E
:100C900000BF00BF2A48006840F48020284908604F
:100CA00000BF00BF4046FFF7F1FA00BF00BF44E0BD
:100CB00000BF00BFFFF7E6FA804600BF00BF4FF05D
:100CC000E020006940F001004FF0E021086100BF22
:100CD00000BF4046FFF7DAFA00BF00BF2DE04FF03B
:100CE000E0204068401C102101EB4010C7B2BC421C
:100CF00022DAA4F11000C11700EBD161C1F347154E
:100D0000C11700EBD1614911A0EB4111CEB200BF78
:100D100000BFFFF7B7FA804600BF00BF0120B04018
:100D2000A90001F1E021C1F8000100BF00BF404669
:100D3000FFF7ACFA00BF00BF00BF00BFBDE8F08105
:100D400024ED00E010B5002400BF00BFFFF79AFAC1
:100D5000044600BF00BF1021054800F0C9FA00BFDB
:100D600000BF2046FFF792FA00BF00BF10BD000091
:100D70005801002010B5FFF7E5FF10BD2DE9F04147
:100D800005460C46002714B900BF00F029F81DB92C
:100D90000A202080BDE8F0811021284601F0D8FF0C
:100DA0000646102E15D200BF00BFFFF76BFA0746AC
:100DB00000BF00BF10222946084801F0A6FF00BF6F
:100DC00000BF3846FFF762FA00BF00BF0020208056
:100DD00002E04FF47A70208000BFDBE7580100206A
:100DE00000BFFEE710B500200249086000F00AF8D5
:100DF00010BD00000000002001490860704700009D
:100E00000000002010B50A48006840F080700849D2
:100E100008600020074948600846006840F001006B
:100E20000860FFF729FE04462046FFF7E5FF10BDE6
:100E3000FCED00E0001000E02DE9F041ADF51C7D77
:100E400004460D461646202194A8FFF7BCFA14214B
:100E50008FA8FFF7B8FA2948006818B90120274978
:100E6000086005E06FF001000DF51C7DBDE8F08124
:100E70000CB105B126B9002020490860401EF3E7F7
:100E800001A804F06AFB9DF8080000909DF8093065
:100E9000BDF80A201AA194A804F0DEFF322294A91A
:100EA00004A806F06DFD074627B10020134908602D
:100EB000401ED9E79DF8050000909DF806309DF88A
:100EC000072015A18FA804F0C7FF8FA8FFF7A2FA8B
:100ED0008046334642468FA904A806F083FF334676
:100EE0002A46214604A806F07DFF04A805F0E2FF8B
:100EF00000200249086000BFB6E700004C01002056
:100F00002F6C6F672F25642D25642D25645F727506
:100F10006E2E6C6F67000000253032643A25303247
:100F2000643A25303264090002F001031BB1D0F8A5
:100F300000340B4302E0D0F800348B43C0F8003497
:100F400002F002031BB1D0F820340B4302E0D0F8CA
:100F500020348B43C0F8203470470000F0B55F4D5B
:100F60002D685F4E35405F4EB5421AD0002416E022
:100F70000125A5400D4085B1D0F8C45F6700032668
:100F8000BE40B543C0F8C45FD0F8C45F6700C2F389
:100F90004116BE403543C0F8C45F651CECB2082C56
:100FA000E6DB02F001051DB1D0F800550D4302E06B
:100FB000D0F800558D43C0F8005502F002051DB170
:100FC000D0F804550D4302E0D0F804558D43C0F825
:100FD000045502F004051DB1D0F808550D4302E098
:100FE000D0F808558D43C0F8085502F008051DB12A
:100FF000D0F818550D4302E0D0F818558D43C0F8CD
:101000001855364D2D68364E3540364EB5420BD00C
:1010100002F010051DB1D0F83C550D4302E0D0F8A8
:101020003C558D43C0F83C5503F001051DB1D0F887
:101030000C550D4302E0D0F80C558D43C0F80C550B
:1010400003F002051DB1D0F810550D4302E0D0F8B1
:1010500010558D43C0F8105503F004051DB1D0F8AC
:1010600014550D4302E0D0F814558D43C0F81455C3
:1010700003F008051DB1D0F81C550D4302E0D0F86F
:101080001C558D43C0F81C55144D2D68144E354029
:10109000144EB54217D003F400751DB1D0F8445575
:1010A0000D4302E0D0F844558D43C0F8445503F495
:1010B00040751DB1D0F840550D4302E0D0F84055C1
:1010C0008D43C0F840551BB9D0F828550D4302E0B8
:1010D000D0F828558D43C0F82855F0BD00E00F40EA
:1010E0000000FF700000051010B50146C1F3074075
:1010F0000F4BDB6E01248440234033B1012303EB0B
:1011000040030C4C54F8230003E04300094C54F80E
:101110002300C1F30722D0F82C350F249440A343B9
:1011200001F00F0494402343C0F82C3510BD00009B
:1011300000E00F40E08E000030B504460D4602226C
:1011400029462046FFF7F0FE0923012229462046C2
:10115000FFF704FF30BD30B504460D460222294694
:101160002046FFF7E1FE0823012229462046FFF72B
:10117000F5FE30BD30B504460D4602222946204614
:10118000FFF7D2FE0823012229462046FFF7E6FE9C
:1011900030BD002303EB8103C2507047014648680D
:1011A00000F0010008B1012070470020FCE7416019
:1011B000704701468868704781607047016A41F056
:1011C0001001016270470246516801F0010008B148
:1011D0000020704701F0120010B101F01C00F8E788
:1011E0000020F6E770B503460C4616461846FFF792
:1011F000E5FF012E01D10F4A00E00F4A142000FB49
:101200000240401E02EB82018900B0FBF1F0451E56
:10121000DD60D3F8C00F00F0010048B1074820445A
:10122000401E0649B0FBF1F0451E45F08000D86035
:1012300070BD0000801A0600A086010080473701BB
:1012400042EA410303607047016A41F020010162F4
:101250000121C0F80418704700B502460B4610463D
:10126000FFF7F2FFC2F8003800BD0000042806D1E5
:101270001949096841F48031174A11602BE00528AB
:1012800006D11549096841F40031134A116022E082
:10129000062806D11049096841F480210E4A1160E0
:1012A00019E00F2808D14FF0E021096941F002014F
:1012B0004FF0E02211610EE010280CD3A0F11001D4
:1012C00001F01F0201219140A0F110025209034BCD
:1012D00053F822201160704724ED00E02C900000AC
:1012E00010B5FEF79EFF08B1012010BD0020FCE7FD
:1012F00030B505460C4622460021284600F026F867
:1013000030BD00000D480E490160014641600021DA
:101310008160C160016141618161C16101620163FC
:10132000C162416207498163C1634FF48061016416
:1013300041640146044A11607047000068010020C2
:1013400048454150B0010020040000202DE9F04143
:1013500003460C4617460FB9BDE8F08103B9FBE719
:101360000025002202E02D022543521C042AFAD354
:10137000384603F0030C1946BCF1000F08D0624652
:1013800003E001F8014B401E521C08B1042AF8D3B7
:101390000E4601E020C6001F0428FBD2314602E0C1
:1013A00001F8014B401E0028FAD100BFD4E700002D
:1013B0001D481E481E481F481F48204820482148F5
:1013C00021482248224823482348244824482548C5
:1013D0002548264826482748274828482848294895
:1013E00029482A482A482B482B482C482C482D4865
:1013F0002D482E482E482F482F4830483048314835
:101400003148324832483348334834483448354804
:1014100035483648364837483748384838483948D4
:10142000394800BF704700007C91000080910000A7
:101430008691000088910000849100008A9100004C
:101440008C9100008E91000090910000929100001C
:101450009491000096910000989100009A910000EC
:101460009C9100009E910000A0910000A2910000BC
:10147000A4910000A6910000A8910000AA9100008C
:10148000AC910000AE910000B0910000B29100005C
:10149000B4910000B6910000B8910000BA9100002C
:1014A000BC910000BE910000C0910000C2910000FC
:1014B000C4910000C6910000C8910000CA910000CC
:1014C000CC910000CE910000D2910000D491000098
:1014D000D6910000D8910000601B0020E01F002082
:1014E000DC910000DE910000E0910000E29100003C
:1014F000E4910000E6910000E8910000EA9100000C
:10150000EC910000DA910000EE9100002DE9F0412D
:1015100005460E46144600271148007818B11220DF
:101520002070BDE8F0812878012808D0022807D073
:10153000032802D0042804D100E000BF00BF00BF90
:1015400002E001202070ECE700BFFEF7C7FE07466F
:101550006E613846FEF7C6FE0020207000BFE0E74F
:101560002500002010B500F019F801F0AFF801F0E7
:10157000DBF801F0FBF801F079F801F039F801F03F
:101580008FF901F0B9F901F031F901F057F900F0E4
:10159000FFFD00F01FF8FFF70BFF10BD0948802189
:1015A00002E0491E002204C00029FAD1064A074B76
:1015B0001A601A46126822F007021A600022044BD1
:1015C0001A80704720200020202200207000002078
:1015D000740000207047000010B50024FEF77EFE66
:1015E000044608480078012808D107480078FF28F9
:1015F00004D205480078401C034908702046FEF7D5
:1016000071FE10BD320000202500002010B500241E
:101610001A480078012830D1FEF760FE04461848C9
:10162000007820B116480078401E1549087014480B
:101630000078F8B913480078E0B901F0BFF9124812
:101640001249097850F82100114908600F480078C4
:101650001049097888420DD00D480068C06B401CC5
:101660000B490968C8630C480068401C0A490860B7
:10167000FEF754FE2046FEF735FE10BD3200002076
:101680002500002026000020F8110020280000205E
:1016900040000020270000200C00002010B500248E
:1016A0000B480078012811D1FEF718FE04460948BE
:1016B000007840B908480078FF2804D2064800782E
:1016C000401C054908702046FEF70CFE10BD0000C6
:1016D00032000020250000202600002010B5002444
:1016E00013480078012821D1FEF7F8FD044611487F
:1016F0000078C0B91048007888B10F480078401EC3
:101700000D4908700846007828B92046FEF7EAFD22
:1017100001F01AF90AE02046FEF7E4FD06E0204653
:10172000FEF7E0FD02E02046FEF7DCFD10BD000004
:1017300032000020250000202600002070B505465C
:1017400000261048007808B1002070BDFEF7C6FDE5
:1017500006460D480468006820B10B4800684068E0
:10176000094908603046FEF7BDFD4CB103202070EA
:1017700025810020606005A06061204600F02AFFFE
:101780002046E2E725000020100000203F00000076
:101790002DE9F04105460E46144600272878032817
:1017A00003D001202070BDE8F0813248007810B1EC
:1017B00002202070F7E73048007810B10D2020702B
:1017C000F1E7FEF78BFD0746288940B12889401EC6
:1017D00028813846FEF786FD00202070E3E7274881
:1017E000006890F8340040F001002449096881F84D
:1017F000340000202149096881F835001F4800683D
:101800000663284600F0A8FE3846FEF76BFD01F09F
:101810009BF8FEF763FD07461848006890F835000E
:1018200020B1012809D0022806D102E00020207052
:101830000BE00E20207008E000BF29460F4800682A
:1018400000F056FE0A20207000BF00BF00200B49A8
:10185000096881F834000949096881F835000749A9
:101860000968C8610549096808623846FEF73AFD0B
:1018700000BF98E725000020260000203800002047
:1018800070B5044600252078032801D0012070BDE2
:10189000FEF724FD0546A07A60B100230122194617
:1018A000204600F0DDFD2846FEF71CFD01F04CF857
:1018B0000020ECE720894FF6FF71884207D220898B
:1018C000401C20812846FEF70DFD0020DFE728465A
:1018D000FEF708FD3320DAE710B50B48007890B921
:1018E00001F06CF80948007809490870094807496F
:1018F000097850F82100084908600846006807493F
:101900000860FEF7F2FC10BD320000202800002025
:1019100027000020F811002040000020380000209F
:1019200010B50024022000F035FBFEF7D7FC04467A
:1019300000200B4908602046FEF7D4FC642000F02C
:1019400029FBFEF7CBFC0446054800680549086002
:101950000120054908702046FEF7C4FC10BD0000B8
:10196000340000201C0000202400002010B5044694
:101970002046FEF7EEFD10BD2DE9F04F85B0814603
:101980008A4693461C46DDE90F78129D002003909D
:10199000FEF7A4FC03902348007830B10398FEF7CB
:1019A000A1FC3C2005B0BDE8F08F1F4850F8240092
:1019B00088BB01201C4941F824000398FEF792FCE3
:1019C0002A464146384601F03DF92B465A465146D3
:1019D000484600F073F904901198CDE90080029513
:1019E0003A4620460E9B049900F0FEFF064636B9A3
:1019F0000E48007801280CD100F0A6FF09E0FEF7A0
:101A00006DFC03900020084941F824000398FEF77C
:101A100069FC3046C6E7FFE70398FEF763FC282021
:101A2000C0E7000025000020F8110020320000204F
:101A300010B504462046FEF78DFD10BD2DE9F0419E
:101A4000054600274A48007810B14020BDE8F081E3
:101A50003F2D01D13E20F9E7FEF740FC0746FF2D60
:101A600003D14448006890F83650434850F8254068
:101A700024B93846FEF736FC4320E7E7012C04D1B1
:101A80003846FEF72FFC3D20E0E714F8380F3B49BD
:101A9000085C617888432178384A505414F8380932
:101AA0001146085C30B994F83A10354800788843FC
:101AB00033490870E06918B12046E16900F018FD6B
:101AC000206A18B12046216A00F029FDA66A16B1E5
:101AD000304600F0B9FD0020206384F8340084F81B
:101AE000350028480078FF2804D226480078401C9A
:101AF000244908703846FEF7F5FB00F0AFFCFEF70E
:101B0000EDFB07461F48007820B11E480078401EB4
:101B10001C490870204600F041F81B480078401E20
:101B2000194908700020144941F82500A06930B90E
:101B300000206169886115496069086005E0D4E9A1
:101B400005014861D4E905108861114800686061A9
:101B50000F4804600FA020653846FEF7C3FB0E480F
:101B60000078012801D100F0EFFE00206EE70000B0
:101B70002500002038000020F81100202A00002055
:101B8000290000202600002033000020440000200F
:101B90003C0000203F0000003200002010B5044649
:101BA0002046FEF7D8FC10BD10B5FEF7D5FC10BDE1
:101BB0002DE9F04106460F4614464FF0000815483F
:101BC000007818B112202070BDE8F081FEF786FB86
:101BD0008046FF2E03D11048006890F836600F4809
:101BE00050F826502DB94046FEF77CFB432020706C
:101BF000EAE7012D05D14046FEF774FB4320207033
:101C0000E2E72F654046FEF76DFB0020207000BF25
:101C1000DAE700002500002038000020F81100203D
:101C200010B504462046FEF798FC10BD10B5FEF72F
:101C300095FC10BD2DE9F04707460D464FF0000A10
:101C4000002028606860FEF749FB8246FF2F03D121
:101C50001848006890F83670174850F827402CB99B
:101C60005046FEF73FFB4320BDE8F087012C04D12E
:101C70005046FEF737FB4320F6E7207C00F00100DA
:101C800020B95046FEF72EFB4520EDE70026D4F89C
:101C90000C90D4F808805046FEF724FB00E0761C38
:101CA00058F8041B0029FAD02E60A9EB06006860E2
:101CB0000020D9E738000020F811002070B5044654
:101CC000101D20F007004FF08076051F28462E607B
:101CD000051F28462C60684E051F28462E604FF0D1
:101CE0001236051F28462E604FF00336051F284682
:101CF0002E604FF00236051F28462E607610051F15
:101D000028462E60051F284629604FF01136051F12
:101D100028462E604FF01036051F28462E604FF0E3
:101D20000936051F28462E604FF00836051F284645
:101D30002E604FF00736051F28462E604FF00636FE
:101D4000051F28462E604FF00536051F28462E60D9
:101D50004FF00436051F28462E6003F00405002DC1
:101D60007ED0F605051F28462E60444E051F2846E6
:101D70002E60434E051F28462E60424E051F284602
:101D80002E60414E051F28462E60404E051F2846F6
:101D90002E603F4E051F28462E603E4E051F2846EA
:101DA0002E603D4E051F28462E603C4E051F2846DE
:101DB0002E603B4E051F28462E603A4E051F2846D2
:101DC0002E60394E051F28462E60384E051F2846C6
:101DD0002E60374E051F28462E60364E051F2846BA
:101DE0002E604FF08346051F28462E60324E051F99
:101DF00028462E60314E051F28462E60304E051FA6
:101E000028462E602F4E051F28462E602E4E051F99
:101E100028462E602D4E051F28462E602C4E051F8D
:101E200028462E604FF08246051F28462E60294E18
:101E3000051F28462E60284E051F28462E60274E77
:101E4000051F28462E604FF08146051F28462E604C
:101E5000234E051F28462E603602051F284600E047
:101E600009E02E604FF07E56051F28462E600026A2
:101E7000051F28462E6070BD512B00000000F84160
:101E80000000F0410000E8410000E0410000D841BE
:101E90000000D0410000C8410000C0410000B8412E
:101EA0000000B0410000A8410000A041000098419E
:101EB0000000904100008841000070410000604136
:101EC000000050410000404100003041000020412E
:101ED000000010410000E0400000C0400000A040B1
:101EE000000040402DE9F04105464FF00008FEF7A4
:101EF000F5F98046FF2D05D12048006890F836504E
:101F0000012608E01D48006890F83600A84201D17B
:101F1000012600E000261A4850F825402CB940461A
:101F2000FEF7E0F94820BDE8F081012C04D14046DD
:101F3000FEF7D8F94320F6E794F838701148C05DF1
:101F400094F8391088430F49C8550846C05D30B928
:101F500094F83A100C48007888430B49087094F8BC
:101F6000340040F0080084F834004046FEF7BAF927
:101F7000012E01D100F0E8FC0020D4E73800002059
:101F8000F81100202A0000202900002010B5FEF7DB
:101F9000E6FA10BD70B5054600261748007800B176
:101FA00070BD1648007800B1FAE71DB3FEF796F948
:101FB00006461348006890F838401248005D104902
:101FC000096891F8391088430E4908550846005DA4
:101FD00040B90B48006890F83A100B4800788843E5
:101FE000094908700648006805633046FEF77AF92B
:101FF00000F0AAFC00BFD3E7250000202600002047
:10200000380000202A000020290000202DE9F0419E
:1020100005460E4617461C461248007810B155205A
:10202000BDE8F0811048007808B13220F8E74FF49D
:102030007A7060434FF47A71B0FBF1F14FF4616054
:102040006843C6EB061200EB8200384400EB400206
:10205000C2EBC01001EBC0084046FFF79BFF002019
:10206000DEE70000250000202600002070B50026D5
:1020700000F072F8FEF732F9064631480068401C5D
:102080002F4908603046FEF72DF92E4800780128C8
:1020900053D12D48007820B1012804D0022809D15D
:1020A00003E001250BE0002509E001250120264978
:1020B000087004E0012500202349087000BF00BF1C
:1020C00005B970BD2148046833E0FEF707F90646FC
:1020D000206B50B3206B401E2063206B28BB94F80C
:1020E000340000F0370040B114F8340F00F0C8009D
:1020F000207001206070343C02E0002084F835003C
:1021000094F8340000F0080078B93834A078104909
:10211000097808430E49087020780E49085C6178F8
:10212000084314F838190B4A505464693046FEF7D6
:10213000D9F894F836003F28C7D100BFC1E70000A6
:1021400058000020320000204800002044000020F9
:10215000290000202A00002010B5FEF701FA0648E9
:102160000088401C044908800846008818B10020F7
:10217000088000F003F810BD7400002010B503487B
:102180000068FFF77DFB0446204610BD6800002074
:10219000F8B54FF42071284800F078FB402127481B
:1021A00000F074FB002514E0681C86B205EB850086
:1021B000214901EBC00406EB860001EBC007642057
:1021C0002070002084F82500E7601DA02062681CB4
:1021D00085B20F2DE8D305EB8500174901EBC0044C
:1021E00064202070002084F82500E06014A02062A4
:1021F0000020144908601449088010201349088001
:102200000D48134908600120FFF798FA114908604A
:102210000020FFF793FA104908606A460FA10D48A5
:102220000068FFF773F96A4611A10B480068FFF7D1
:102230006DF900F027F8F8BD601B0020E01F0020BA
:102240003F000000600000205E0000205C000020D5
:102250006C000020640000206800002075432F4FB0
:10226000532D494920546D724C6F636B0000000080
:1022700075432F4F532D494920546D725369676E32
:10228000616C000000B587B00320002180220A4B5A
:10229000CDE90132CDE903104FF6FD703D23074A29
:1022A00000900748FFF768FB06AA06A13D20FFF74C
:1022B0007FFC07B000BD0000E01D0020DC1F0020F7
:1022C0004123000075432F4F532D494920546D720F
:1022D0000000000070B50B46032580F82550012B47
:1022E00005D1154EC5693668354445610CE08569F0
:1022F0002DB9114EC56936683544456104E00E4E6E
:102300008569366835444561057D05F007040B4D48
:1023100005EBC4010D682DB908600025C5600125D5
:102320008D8006E00A680860C26010618D886D1CAF
:102330008D800025056170BD60000020E01F002039
:1023400008B500BF00BF6A4600211A480068FFF7C1
:102350001FFAFFF7A3F918480068401C16490860E7
:102360000846007800F00708144800EBC8073C68EE
:102370001AE0E668104960690968884213D120466E
:1023800000F01EF894F82400022804D10121204610
:10239000FFF7A0FF02E0022084F82500656815B170
:1023A0002046A168A8473446002CE2D1FFF796F9F1
:1023B000C9E700006800002060000020E01F002046
:1023C00030B5057D05F007040D4D05EBC4031D6810
:1023D000854205D1C168196039B100250D6104E05D
:1023E0000169C268CA6002B11161012580F82550F7
:1023F0000025C56005619D886D1E9D8030BD000073
:10240000E01F002010B5FDF769FF0446064800787C
:10241000401C054908702046FDF764FFFFF726FEC3
:10242000FFF7F4F810BD00002500002001464A1E09
:102430004FF0E0235A61084A106820F07F4000BF47
:1024400010601A46126942F005021A611A461269B2
:1024500042F002021A61704720ED00E07047000070
:102460002DE9F04F05460F4690469946A87A1C493B
:102470000E5C05F10B00805D11F800B00BEBC6009F
:1024800000F0FF0A174850F82A4000202434E0608A
:102490002760207C20EA0800207484F81190207CBA
:1024A000243C00F0080068B994F83A000E49097815
:1024B00008430D4908700D48805D94F839100843B1
:1024C0000A4988552946204600F012F8206A20B1B2
:1024D0002046216A00F023F8E5615046BDE8F08F00
:1024E0007C900000F8110020290000202A00002024
:1024F00010B590F8382001F10B039B5C90F839403F
:10250000A34301F10B04A35423469B5C23B98B7AAC
:1025100090F83A40A3438B720023C36110BDF0B51D
:10252000024612F8384F95785678383A0B461868B4
:102530000FE000F10B073F5DB74300F10B0C0CF807
:10254000047067463F5D17B9877AAF4387721B1DDA
:1025500018680028EDD1F0BD10B51B4A1268D06193
:10256000194A126892F8383000F10B02D25C164B0F
:102570001B6893F839301A43134B1B6893F83840A3
:1025800000F10B031A55827A0F4B1B6893F83A300F
:102590001A4382720C4A126892F838100B4A525C45
:1025A000094B1B6893F839309A43084B5A541A4622
:1025B000525C42B9044A126892F83A30044A1278DE
:1025C0009A43034B1A7010BD380000202A000020E7
:1025D00029000020014600228A72002005E0002325
:1025E00001F10B021354421CD0B20828F7D37047F4
:1025F0002DE9F041A021114800F048F900250DE037
:10260000681C86B20D4800EB051400EB061700208D
:10261000207067600AA0E060681C85B2092DEFD3C6
:10262000064800EB051400202070606004A0E06004
:10263000024804490860BDE8F0810000580D002000
:102640003F0000001400002030B501464A680868C9
:102650002AB9CC68606028B10025456002E01060AE
:1026600000B142608B6800259D6230BD70B54FF4AB
:10267000BD61134800F00AF9002411E0601C85B226
:1026800004EB44000E4901EBC00305EB450001EBF0
:10269000C006002018705E600AA05861601C84B2F9
:1026A0003E2CEBD304EB4400054901EBC0030020B2
:1026B0001870586003A0586108460349086070BD4F
:1026C000700700203F0000001000002000200B4990
:1026D00008600B4908700B4908700B4908700B49DA
:1026E00008700B4908600B4908600B4908600B49EA
:1026F00008600B4908700B490870704758000020AB
:102700002500002026000020330000203200002099
:102710000C00002034000020200000201C000020BD
:10272000240000205400002000210A4A11700020DB
:1027300004E00021084A1154411CC8B20828F8D30B
:102740000021064A1170064A1170064A1160064AB5
:1027500011607047290000202A0000202700002077
:1027600028000020400000203800002070B54FF401
:10277000F261194800F08AF84FF48071174800F0B0
:1027800085F8002413E0601CC5B204EB440000EBA4
:10279000C400114901EBC00305EB450000EBC50087
:1027A00001EBC0065E610EA01865601CC4B2152C5A
:1027B000E9D304EB440000EBC400074901EBC0037C
:1027C0000020586106A018650020064908600248EC
:1027D0000549086070BD0000F8120020F8110020C3
:1027E0003F000000440000203C00002000B587B0FE
:1027F0000320002180220A4BCDE90132CDE90310EC
:102800004FF6FF703F23074A00900748FFF7B4F8E0
:1028100006AA06A13F20FFF7CBF907B000BD0000D4
:10282000F80F0020F4110020292B000075432F4FD2
:10283000532D49492049646C6500000000B587B0FC
:102840000320002180220A4BCDE90132CDE903109B
:102850004FF6FE703E23074A00900748FFF78CF8BA
:1028600006AA06A13E20FFF7A3F907B000BD0000AD
:10287000F80D0020F40F0020692B000075432F4F46
:10288000532D4949205374617400000004E0002274
:1028900000F8012B4A1E91B20029F8D170470000C0
:1028A00070B578211148FFF7F1FF00240EE004EB2A
:1028B00044000E4901EBC005601C00EB400001EB39
:1028C000C00068600AA06861601C84B2042CEED36A
:1028D00004EB4400054901EBC0050020686004A03A
:1028E000686108460349086070BD0000881A00202E
:1028F0003F0000004C0000202DE9F041602110480D
:10290000FFF7C4FF00240DE0601C86B204EB440016
:102910000B4901EBC00506EB460001EBC0072F6039
:10292000601C84B2032CEFD304EB4400044901EB98
:10293000C00500202860084602490860BDE8F08113
:10294000001B00205000002010B50024FDF7C6FC3D
:10295000044613480078F8B912480078E0B900F04E
:102960002DF811481149097850F8210010490860E4
:102970000E4800780F49097888420DD00C4800684D
:10298000C06B401C0A490968C8630B480068401CBA
:1029900009490860FDF7BDFC2046FDF7A3FC10BD0A
:1029A0002500002026000020F8110020280000202B
:1029B00040000020270000200C0000200649074AA4
:1029C0001278885C0649095C034A515C01EBC0013E
:1029D000044A1170704700007C900000290000201C
:1029E0002A000020280000202DE9F84F05460F4658
:1029F00090469946DDE90AAB00200090FDF76EFC99
:102A0000009042480468002C7BD01C3454F8080C19
:102A10003E4908600098FDF765FC44F81C7CA576EB
:102A2000002020766076606144F818BC44F810AC51
:102A300044F8148C0C9824F80C0C24F80A9C002000
:102A4000E077E810207705F00700E076217F01208D
:102A50008840A077E17E01208840607700202060D8
:102A60006060E060A0602062A0626062E06220635B
:102A700027A060631C3C002606E0002104F15400FE
:102A800040F82610701CC6B2002EF6D02046FEF785
:102A90006DFFFDF723FC00901E4840F8254000988C
:102AA000FDF720FC2046FEF7C3FFFDF717FC009062
:102AB0001948006860610020A0611748006810B1E3
:102AC000154800688461144804603834A0781349BC
:102AD000097808431149087020781149085C617829
:102AE000084314F838190E4A50540E480078401C18
:102AF0000C4908700098FDF7F5FB0020BDE8F88F41
:102B0000FFE70098FDF7EEFB4220F7E73C000020CE
:102B10003F000000F81100204400002029000020A0
:102B20002A00002033000020002400BF00BFFDF772
:102B3000D5FB044605480068401C0449086020464F
:102B4000FDF7D0FBFFF730F8F1E70000340000207C
:102B500010B504480068FFF763F8FF20FEF76EFF2A
:102B600010BD00003800002000BF00BF02E0C820F8
:102B7000FFF710FA1F4800780028F8D01E480068B8
:102B80006421B0FBF1F01C4908600846006828B9D0
:102B900000201A490870FF20FFF7A4F9FDF79EFBFB
:102BA00004461548006864214843154908602046DA
:102BB000FDF798FB00BFFDF791FB04461048006845
:102BC0001049086000200E4908602046FDF78AFB86
:102BD0000C48006808490968B0FBF1F0C0F16400D6
:102BE00006490870FFF722F800F00EF86420FFF79E
:102BF000D1F9E0E7240000201C000020180000208C
:102C000034000020200000207CB5002514E0694637
:102C10002846FFF70FF8064666B9094850F82540E0
:102C200044B1012C06D0D4E9020100EB8100A0647C
:102C30000198E064681CC5B23F2DE8D97CBD000056
:102C4000F811002002F0010343B102F002032BB19E
:102C500002E0491E002308C00029FAD1704701464E
:102C6000C868C0F3001070472DE9F04F0C461D46B0
:102C7000DDE909C815B94FF0000A01E04FF0040A78
:102C800057464760B4FBFCF6002100BF891CB6FB29
:102C9000F1FAAAF10103FF2BF8D801614FEA827A19
:102CA0004FEA1A6902F0300249EA032A4AEA020AA4
:102CB000A8F1010B4AEA0B070760BDE8F08F00BFDF
:102CC000C26802F00402002AFAD082680A607047E3
:102CD0000246D06800F0040018B190680860012036
:102CE00070470020FCE700BFC26802F00202002A21
:102CF000FAD081607047416821F00201416070475D
:102D0000416841F002014160704770B504460D46CC
:102D100016460CB9002070BD0DB90020FBE7214616
:102D20002A46002304E010780870491C521C5B1CE2
:102D300021B11AB1107808B1B342F4D301B10AB984
:102D40000020E8E7B34201D2002008702046E2E705
:102D500010B502460B461146002001E0491C401CFC
:102D600019B10C780CB19842F8D310BD10B50121FF
:102D7000C0F30722094B1A4402F0704242F000727D
:102D8000C0F30723054C2344C3F3130342EA431261
:102D9000C3B242EA8302116010BD000000E60F409A
:102DA00001480068704700000800002010B507A027
:102DB00000F03AF80849086008A000F035F80B491F
:102DC000086002F005FC044610BD00005461736BFE
:102DD00052746353796E6300380100205461736B41
:102DE000527463416C61726D00000000300100207C
:102DF00010B54FF47A71002002F086F801210846E0
:102E000002F082F802A000F00FF80449086010BD3B
:102E10005461736B54696D65720000002C010020D1
:102E200010B502F001FA10BD70B5054615B94FF0A6
:102E3000FF3070BD002425E004EB0410144901EBC1
:102E40004000407801281BD0002004EB0411104AF8
:102E500002F81100012004EB041102EB410148705B
:102E60002846FDF7D7FA064604EB0411084A02EBA0
:102E70004101881C32462946FDF78CFA2046D8E7E6
:102E8000601C44B2142CD7DB4FF0FF30D1E70000B8
:102E9000B8240020C26840F201139A43C2600A0EAF
:102EA0000260114A1268114B1A40114B9A4211D11B
:102EB000CAB201F4702342EA131242F40072426073
:102EC00001F47002C1F3072343EA122242F40072B4
:102ED000826008E0CAB242F400724260C1F3072285
:102EE00042F400728260704700E00F400000FF7003
:102EF00000000A10C26840F201130B401A43C2607E
:102F000070474162704782690A4382617047CBB261
:102F100003B1826201F47F4303B1C26270478168EA
:102F200041F00101816070470121C16070470121BA
:102F3000C0F8001C704701607047816841F00201D1
:102F4000816070470149C0F8001C704751E5CC1AF8
:102F50002DE9F04104460D4616461F46082C03DBBA
:102F60004FF0FF30BDE8F08104EB4400EB4911F86D
:102F7000200010B94FF0FF30F4E704EB4400E749BC
:102F800001EB80004078012801D10020EAE714BB62
:102F9000E348FFF7EBFEE348FFF7E8FEE148FFF701
:102FA000E5FEE148FEF7A0F8E048FEF79DF80421B1
:102FB000DF48FEF7D0F80821DD48FEF7BDF8A6B9D6
:102FC000DC48854208D1FFF7EBFE804600224146EF
:102FD000D948FEF707F90CE0FFF7E2FE8046012230
:102FE0004146D548FEF7FEF803E03946D248FEF7E1
:102FF00033F9012C33D1CA48401CFFF7B7FEC9484A
:10300000401DFFF7B3FEC748401DFFF7AFFECB489A
:10301000FEF76AF8CA48FEF767F80121C948FEF7CB
:103020009AF80221C748FEF787F8A6B9C148854239
:1030300008D1FFF7B5FE804600224146C248FEF7A0
:10304000D1F80CE0FFF7ACFE804601224146BE48B5
:10305000FEF7C8F803E03946BB48FEF7FDF8022C3E
:1030600033D1AF48801CFFF781FEAE480930FFF72F
:103070007DFEAC480930FFF779FEB448FEF734F81E
:10308000B348FEF731F80221B248FEF764F8012197
:10309000B048FEF751F8A6B9A648854208D1FFF717
:1030A0007FFE804600224146AB48FEF79BF80CE0CD
:1030B000FFF776FE804601224146A748FEF792F8C8
:1030C00003E03946A448FEF7C7F8032C33D19448EF
:1030D000C01CFFF74BFE93480830FFF747FE9148AE
:1030E0000830FFF743FE9D48FDF7FEFF9C48FDF7C3
:1030F000FBFF10219B48FEF72EF820219948FEF790
:103100001BF8A6B98B48854208D1FFF749FE8046D7
:10311000002241469448FEF765F80CE0FFF740FEB8
:103120008046012241469048FEF75CF803E03946AC
:103130008D48FEF791F8042C33D17948001DFFF734
:1031400015FE78480830FFF711FE76480830FFF783
:103150000DFE8648FDF7C8FF8548FDF7C5FF4021F5
:103160008048FDF7F8FF80217E48FDF7E5FFA6B90E
:103170007048854208D1FFF713FE80460022414681
:103180007C48FEF72FF80CE0FFF70AFE804601228C
:1031900041467848FEF726F803E039467548FEF7C1
:1031A0005BF8052C31D15E48401DFFF7DFFD5D481F
:1031B000FFF7DCFD5B48FFF7D9FD6F48FDF794FF93
:1031C0006E48FDF791FF01215948FDF7C4FF022128
:1031D0005748FDF7B1FFA6B95648854208D1FFF719
:1031E000DFFD8046002241466548FDF7FBFF0CE00D
:1031F000FFF7D6FD8046012241466148FDF7F2FF08
:1032000003E039465E48FEF727F8062C37D14448DC
:10321000801DFFF7ABFD4348401EFFF7A7FD414867
:10322000401EFFF7A3FD41F60200FDF75DFF41F6EA
:103230000240FDF759FF40214FF04020FDF78BFF82
:1032400080214FF04020FDF777FFA6B9394885422D
:1032500008D1FFF7A5FD8046002241464948FDF709
:10326000C1FF0CE0FFF79CFD804601224146454826
:10327000FDF7B8FF03E039464248FDF7EDFF072CA4
:1032800033D12748C01DFFF771FD2648801CFFF78A
:103290006DFD2448801CFFF769FD3B48FDF724FFC6
:1032A0003A48FDF721FF01213948FDF754FF02217B
:1032B0003748FDF741FFA6B91E48854208D1FFF700
:1032C0006FFD8046002241463248FDF78BFF0CE03F
:1032D000FFF766FD8046012241462E48FDF782FF3A
:1032E00003E039462B48FDF7B7FF012004EB44010A
:1032F0000A4A02EB8101487004EB4400114601EBDD
:103300008000456004EB440001EB8000067204EB92
:10331000440001EB80004772002023E67800002083
:10332000002000F0010800F002080100020C01007A
:1033300000500040A086010000000240020006008C
:1033400002040600006002400010024002040A006D
:1033500002000A000020064000200240021009007E
:103360000214090000100640003002400218090053
:10337000021C090000000C400200010002040100D0
:1033800000100C4000200C40020003000204030067
:103390000070004000300C402DE9F047054688469B
:1033A00017461E464FF00009082D03DB4FF0FF3093
:1033B000BDE8F08767B105EB4500F84911F820003A
:1033C00030B12EB105EB450001EB8000407810B91B
:1033D0004FF0FF30ECE702E00A20FEF7DBFD05EBE3
:1033E0004500EE4901EB8000807A0128F4D00120ED
:1033F00005EB4501E94A02EB81018872FCF76EFF9B
:10340000814605EB4500E54901EB8000007A002884
:103410006FD1002D6ED102E00120FEF7BBFDE04828
:10342000FDF7BCFE0028F7D101224146DC48FDF73C
:1034300007FF012E2BD10721D948FDF7B8FED84848
:10344000FDF7C1FE58B14846FCF74CFF002005EBE4
:103450004501D24A02EB81018872401EA8E702E0D2
:103460000120FEF797FDCE48FDF798FE0028F7D122
:10347000CB48FDF79EFE38704846FCF733FF00202E
:1034800005EB4501C54A02EB8101887290E70024F3
:103490003FE024B90B21C248FDF789FE0BE0701E06
:1034A000A04204D10521BE48FDF781FE03E00921B9
:1034B000BB48FDF77CFEBA48FDF785FED8B1701E0B
:1034C000A0420AD0B648FDF77EFE00F0100010289A
:1034D00003D00421B248FDF76AFE4846FCF702FF1C
:1034E000002005EB4501AD4A02EB81018872401EC8
:1034F0005EE722E210E002E00120FEF74BFDA84863
:10350000FDF74CFE0028F7D1A548FDF752FE3855CF
:10351000641CB442BDD3A3E3012D7FD102E001209E
:10352000FEF738FD9F48FDF739FE0028F7D101224C
:1035300041469C48FDF784FE012E2BD10721994876
:10354000FDF735FE9748FDF73EFE58B14846FCF7BB
:10355000C9FE002005EB4501904A02EB810188720B
:10356000401E25E702E00120FEF714FD8D48FDF71F
:1035700015FE0028F7D18B48FDF71BFE3870484632
:10358000FCF7B0FE002005EB4501844A02EB810107
:1035900088720DE700243EE024B90B218148FDF735
:1035A00006FE0BE0701EA04204D105217D48FDF708
:1035B000FEFD03E009217B48FDF7F9FD7948FDF7A1
:1035C00002FEC8B1701EA0420AD07648FDF7FBFD8E
:1035D00000F01000102803D004217248FDF7E7FD29
:1035E0004846FCF77FFE002005EB45016B4A02EBE5
:1035F00081018872401EDBE603E00FE00120FEF748
:10360000C9FC6848FDF7CAFD0028F7D16548FDF7F9
:10361000D0FD3855641CB442BED321E3022D7FD1C6
:1036200002E00120FEF7B6FC5F48FDF7B7FD002879
:10363000F7D1012241465C48FDF702FE012E2BD155
:1036400007215948FDF7B3FD5748FDF7BCFD58B1B8
:103650004846FCF747FE002005EB45014F4A02EBC8
:1036600081018872401EA3E602E00120FEF792FC71
:103670004D48FDF793FD0028F7D14B48FDF799FD24
:1036800038704846FCF72EFE002005EB4501434A02
:1036900002EB810188728BE600243EE024B90B2105
:1036A0004148FDF784FD0BE0701EA04204D10521C6
:1036B0003D48FDF77CFD03E009213B48FDF777FD20
:1036C0003948FDF780FDC8B1701EA0420AD03648C7
:1036D000FDF779FD00F01000102803D004213248D6
:1036E000FDF765FD4846FCF7FDFD002005EB4501B3
:1036F0002A4A02EB81018872401E59E603E00FE07E
:103700000120FEF747FC2848FDF748FD0028F7D1C7
:103710002548FDF74EFD3855641CB442BED39FE2E8
:10372000032D77D102E00120FEF734FC1F48FDF79E
:1037300035FD0028F7D1012241461C48FDF780FDE8
:10374000012E35D107211948FDF731FD1748FDF746
:103750003AFD58B14846FCF7C5FD002005EB450190
:103760000E4A02EB81018872401E21E602E0012030
:10377000FEF710FC0D48FDF711FD0028F7D10B48AE
:10378000FDF717FD38704846FCF7ACFD002005EB4F
:103790004501024A02EB8101887209E678000020A7
:1037A00000000240001002400020024000300240B1
:1037B00000243EE024B90B21FE48FDF7F8FC0BE0A5
:1037C000701EA04204D10521FA48FDF7F0FC03E089
:1037D0000921F848FDF7EBFCF648FDF7F4FCD0B101
:1037E000701EA0420AD0F348FDF7EDFC00F0100077
:1037F000102803D00421EF48FDF7D9FC4846FCF718
:1038000071FD002005EB4501EB4A02EB8101887256
:10381000401ECDE510E002E00120FEF7BBFBE548CD
:10382000FDF7BCFC0028F7D1E248FDF7C2FC385593
:10383000641CB442BED313E2042D7FD102E0012008
:10384000FEF7A8FBDD48FDF7A9FC0028F7D101220F
:103850004146DA48FDF7F4FC012E2BD10721D74869
:10386000FDF7A5FCD548FDF7AEFC58B14846FCF77E
:1038700039FD002005EB4501CF4A02EB810188723A
:10388000401E95E502E00120FEF784FBCB48FDF7E2
:1038900085FC0028F7D1C948FDF78BFC38704846F5
:1038A000FCF720FD002005EB4501C34A02EB810136
:1038B00088727DE500243EE024B90B21BF48FDF766
:1038C00076FC0BE0701EA04204D10521BB48FDF739
:1038D0006EFC03E00921B948FDF769FCB748FDF724
:1038E00072FCC8B1701EA0420AD0B448FDF76BFC50
:1038F00000F01000102803D00421B048FDF757FC59
:103900004846FCF7EFFC002005EB4501AA4A02EB14
:1039100081018872401E4BE503E00FE00120FEF7B5
:1039200039FBA648FDF73AFC0028F7D1A348FDF77C
:1039300040FC3855641CB442BED391E1052D7FD1C3
:1039400002E00120FEF726FB9D48FDF727FC00283A
:10395000F7D1012241469A48FDF772FC012E2BD186
:1039600007219748FDF723FC9548FDF72CFC58B13B
:103970004846FCF7B7FC002005EB45018E4A02EBF8
:1039800081018872401E13E502E00120FEF702FB70
:103990008B48FDF703FC0028F7D18948FDF709FCA7
:1039A00038704846FCF79EFC002005EB4501824A32
:1039B00002EB81018872FBE400243EE024B90B2174
:1039C0007F48FDF7F4FB0BE0701EA04204D10521F7
:1039D0007B48FDF7ECFB03E009217948FDF7E7FBA5
:1039E0007748FDF7F0FBC8B1701EA0420AD07448BA
:1039F000FDF7E9FB00F01000102803D00421704807
:103A0000FDF7D5FB4846FCF76DFC002005EB4501B2
:103A1000694A02EB81018872401EC9E403E00FE0AD
:103A20000120FEF7B7FA6648FDF7B8FB0028F7D18A
:103A30006348FDF7BEFB3855641CB442BED30FE1AA
:103A4000062D7FD102E00120FEF7A4FA5D48FDF7C4
:103A5000A5FB0028F7D1012241465A48FDF7F0FBAB
:103A6000012E2BD107215748FDF7A1FB5548FDF743
:103A7000AAFB58B14846FCF735FC002005EB450190
:103A80004D4A02EB81018872401E91E402E0012060
:103A9000FEF780FA4B48FDF781FB0028F7D1494833
:103AA000FDF787FB38704846FCF71CFC002005EB4F
:103AB0004501414A02EB8101887279E400243EE02D
:103AC00024B90B213F48FDF772FB0BE0701EA042AA
:103AD00004D105213B48FDF76AFB03E00921394881
:103AE000FDF765FB3748FDF76EFBC8B1701EA042BD
:103AF0000AD03448FDF767FB00F01000102803D00F
:103B000004213048FDF753FB4846FCF7EBFB00204F
:103B100005EB4501284A02EB81018872401E47E40B
:103B200003E00FE00120FEF735FA2648FDF736FBEB
:103B30000028F7D12348FDF73CFB3855641CB442FC
:103B4000BED38DE0072D7AD102E00120FEF722FAE4
:103B50001D48FDF723FB0028F7D1012241461A48F2
:103B6000FDF76EFB012E38D107211748FDF71FFB2B
:103B70001548FDF728FB58B14846FCF7B3FB002079
:103B800005EB45010C4A02EB81018872401E0FE4EF
:103B900002E00120FEF7FEF90B48FDF7FFFA0028CE
:103BA000F7D10948FDF705FB38704846FCF79AFB4A
:103BB00000200BE0003002407800002000000C40A4
:103BC00000100C4000200C4000300C4005EB45017B
:103BD000294A02EB8101887240E400243EE024B9C6
:103BE0000B212648FDF7E3FA0BE0701EA04204D13A
:103BF00005212248FDF7DBFA03E009211F48FDF704
:103C0000D6FA1E48FDF7DFFAD0B1701EA0420AD0E6
:103C10001A48FDF7D8FA00F01000102803D004214C
:103C20001648FDF7C4FA4846FCF75CFB002005EB9C
:103C30004501114A02EB81018872401E0EE40FE03B
:103C400002E00120FEF7A6F90C48FDF7A7FA0028CC
:103C5000F7D10A48FDF7ADFA3855641CB442BED31B
:103C60004846FCF73FFB002005EB4501024A02EB0A
:103C70008101887200BF09E47800002000300C4008
:103C80002DE9F0470546884616461F464FF00009C5
:103C9000082D03DB4FF0FF30BDE8F08766B105EB80
:103CA0004500FA4911F8200030B12FB105EB45006D
:103CB00001EB8000407810B94FF0FF30ECE702E0F4
:103CC0000A20FEF767F905EB4500F04901EB80009B
:103CD000807A0128F4D0012005EB4501EB4A02EB84
:103CE00081018872FCF7FAFA814605EB4500E74945
:103CF00001EB8000007A00287BD1002D7AD102E010
:103D00000120FEF747F9E248FDF748FA0028F7D10D
:103D100000224146DE48FDF793FA012F2BD131787E
:103D2000DB48FDF749FA0721D948FDF740FAD848A2
:103D3000FDF749FA58B14846FCF7D4FA002005EBE4
:103D40004501D24A02EB81018872401EA4E702E0DD
:103D50000120FEF71FF9CE48FDF720FA0028F7D121
:103D60004846FCF7BFFA002005EB4501C74A02EBC5
:103D70008101887290E7002447E044B9315DC4486E
:103D8000FDF71AFA0321C248FDF711FA13E0781E75
:103D9000A04208D1315DBE48FDF70EFA0521BC48AE
:103DA000FDF705FA07E0315DB948FDF705FA012195
:103DB000B748FDF7FCF9B648FDF705FAD8B1781E0B
:103DC000A0420AD0B248FDF7FEF900F0100010281A
:103DD00003D00421AE48FDF7EAF94846FCF782FA21
:103DE000002005EB4501A94A02EB81018872401EC3
:103DF00052E73FE20CE002E00120FEF7CBF8A448D6
:103E0000FDF7CCF90028F7D1641CBC42B5D3D9E347
:103E1000012D79D102E00120FEF7BCF89D48FDF7A5
:103E2000BDF90028F7D1002241469A48FDF708FA6B
:103E3000012F2BD131789748FDF7BEF9072195481E
:103E4000FDF7B5F99348FDF7BEF958B14846FCF7C0
:103E500049FA002005EB45018C4A02EB810188728A
:103E6000401E19E702E00120FEF794F88948FDF7AB
:103E700095F90028F7D14846FCF734FA002005EB05
:103E80004501824A02EB8101887205E7002446E081
:103E900044B9315D7F48FDF78FF903217D48FDF777
:103EA00086F913E0781EA04208D1315D7948FDF70C
:103EB00083F905217748FDF77AF907E0315D754808
:103EC000FDF77AF901217348FDF771F97148FDF7A3
:103ED0007AF9D0B1781EA0420AD06E48FDF773F986
:103EE00000F01000102803D004216A48FDF75FF9A4
:103EF0004846FCF7F7F9002005EB4501634A02EB61
:103F000081018872401EC7E60CE002E00120FEF746
:103F100041F86048FDF742F90028F7D1641CBC4223
:103F2000B6D34FE3022D79D102E00120FEF732F83B
:103F30005948FDF733F90028F7D100224146564889
:103F4000FDF77EF9012F2BD131785348FDF734F975
:103F500007215148FDF72BF94F48FDF734F958B1C7
:103F60004846FCF7BFF9002005EB4501474A02EB44
:103F700081018872401E8FE602E00120FEF70AF8F8
:103F80004548FDF70BF90028F7D14846FCF7AAF998
:103F9000002005EB45013D4A02EB810188727BE67A
:103FA000002446E044B9315D3B48FDF705F90321A3
:103FB0003948FDF7FCF813E0781EA04208D1315DC6
:103FC0003548FDF7F9F805213348FDF7F0F807E02B
:103FD000315D3148FDF7F0F801212F48FDF7E7F892
:103FE0002D48FDF7F0F8D0B1781EA0420AD02A483B
:103FF000FDF7E9F800F01000102803D0042126484E
:10400000FDF7D5F84846FCF76DF9002005EB4501B2
:104010001E4A02EB81018872401E3DE60CE002E080
:104020000120FDF7B7FF1C48FDF7B8F80028F7D1CD
:10403000641CBC42B6D3C5E2032D7CD102E0012052
:10404000FDF7A8FF1548FDF7A9F80028F7D10022D1
:1040500041461248FDF7F4F8012F35D131780F4869
:10406000FDF7AAF807210D48FDF7A1F80B48FDF769
:10407000AAF8A8B14846FCF735F9002005EB450140
:10408000024A02EB81018872401E05E6780000209A
:1040900000000240001002400020024000300240B8
:1040A00002E00120FDF776FFF648FDF777F80028DB
:1040B000F7D14846FCF716F9002005EB4501F24A16
:1040C00002EB81018872E7E5002447E044B9315DE5
:1040D000EC48FDF771F80321EA48FDF768F813E0B2
:1040E000781EA04208D1315DE648FDF765F805214C
:1040F000E448FDF75CF807E0315DE248FDF75CF865
:104100000121E048FDF753F8DE48FDF75CF8D8B12F
:10411000781EA0420AD0DB48FDF755F800F01000E9
:10412000102803D00421D748FDF741F84846FCF792
:10413000D9F8002000E014E005EB4501D24A02EB7B
:1041400081018872401EA7E502E00120FDF722FFF1
:10415000CC48FDF723F80028F7D1641CBC42B5D346
:1041600030E2042D79D102E00120FDF713FFC748AA
:10417000FDF714F80028F7D100224146C348FDF7A7
:104180005FF8012F2BD13178C048FDF715F80721D2
:10419000BE48FDF70CF8BD48FDF715F858B1484684
:1041A000FCF7A0F8002005EB4501B74A02EB8101BE
:1041B0008872401E70E502E00120FDF7EBFEB34877
:1041C000FCF7ECFF0028F7D14846FCF78BF80020FD
:1041D00005EB4501AC4A02EB810188725CE50024E5
:1041E00046E044B9315DA948FCF7E6FF0321A74842
:1041F000FCF7DDFF13E0781EA04208D1315DA34833
:10420000FCF7DAFF0521A148FCF7D1FF07E0315D9B
:104210009E48FCF7D1FF01219C48FCF7C8FF9B4852
:10422000FCF7D1FFD0B1781EA0420AD09748FCF726
:10423000CAFF00F01000102803D004219348FCF7B7
:10424000B6FF4846FCF74EF8002005EB45018E4AC4
:1042500002EB81018872401E1EE50CE002E00120A5
:10426000FDF798FE8948FCF799FF0028F7D1641CF8
:10427000BC42B6D3A6E1052D79D102E00120FDF7BD
:1042800089FE8348FCF78AFF0028F7D100224146C7
:104290007F48FCF7D5FF012F2BD131787C48FCF704
:1042A0008BFF07217A48FCF782FF7948FCF78BFFE8
:1042B00058B14846FCF716F8002005EB4501724A54
:1042C00002EB81018872401EE6E402E00120FDF766
:1042D00061FE6F48FCF762FF0028F7D14846FCF703
:1042E00001F8002005EB4501674A02EB8101887265
:1042F000D2E4002446E044B9315D6548FCF75CFF38
:1043000003216348FCF753FF13E0781EA04208D155
:10431000315D5F48FCF750FF05215D48FCF747FF22
:1043200007E0315D5A48FCF747FF01215848FCF788
:104330003EFF5748FCF747FFD0B1781EA0420AD095
:104340005348FCF740FF00F01000102803D0042170
:104350004F48FCF72CFF4846FBF7C4FF002005EB55
:104360004501494A02EB81018872401E94E40CE049
:1043700002E00120FDF70EFE4548FCF70FFF002884
:10438000F7D1641CBC42B6D31CE1062D79D102E002
:104390000120FDF7FFFD3F48FCF700FF0028F7D1A3
:1043A000002241463B48FCF74BFF012F2BD13178CF
:1043B0003848FCF701FF07213648FCF7F8FE35487E
:1043C000FCF701FF58B14846FBF78CFF002005EBD6
:1043D00045012D4A02EB81018872401E5CE402E037
:1043E0000120FDF7D7FD2B48FCF7D8FE0028F7D1B8
:1043F0004846FBF777FF002005EB4501224A02EB18
:104400008101887248E4002450E044B9315D2148BC
:10441000FCF7D2FE03211F48FCF7C9FE13E0781E0B
:10442000A04208D1315D1B48FCF7C6FE05211948A2
:10443000FCF7BDFE07E0315D1648FCF7BDFE01212B
:104440001448FCF7B4FE1348FCF7BDFE20B3781EF9
:10445000A0420AD00F48FCF7B6FE00F0100010286A
:1044600003D004210B48FCF7A2FE4846FBF73AFFB5
:10447000002005EB4501044A02EB81018872401ED1
:104480000AE416E0003002407800002000000C40F2
:1044900000100C4000200C4002E00120FDF77AFDE6
:1044A0004E48FCF77BFE0028F7D1641CBC42ACD31D
:1044B00088E0072D79D102E00120FDF76BFD484827
:1044C000FCF76CFE0028F7D1002241464448FCF777
:1044D000B7FE012F2BD131784148FCF76DFE072143
:1044E0003F48FCF764FE3E48FCF76DFE58B1484675
:1044F000FBF7F8FE002005EB45013A4A02EB81018B
:104500008872401E22E402E00120FDF743FD34489A
:10451000FCF744FE0028F7D14846FBF7E3FE0020F5
:1045200005EB45012F4A02EB810188720EE400245D
:1045300046E044B9315D2A48FCF73EFE0321284895
:10454000FCF735FE13E0781EA04208D1315D244807
:10455000FCF732FE05212248FCF729FE07E0315D19
:104560001F48FCF729FE01211D48FCF720FE1C48CE
:10457000FCF729FED0B1781EA0420AD01848FCF7FB
:1045800022FE00F01000102803D004211448FCF78C
:104590000EFE4846FBF7A6FE002005EB4501114A3A
:1045A00002EB81018872401E22E40BE002E0012050
:1045B000FDF7F0FC0A48FCF7F1FD0028F7D1641C78
:1045C000BC42B6D34846FBF78DFE002005EB450103
:1045D000044A02EB8101887200BF09E400200C400C
:1045E00000300C40780000207047000010B50F48E4
:1045F000FEF7BCFB012211460D48FCF795FC4FF479
:104600000273012211460A48FCF7A8FC0748FEF78E
:10461000ADFB012202210648FCF786FC4FF4027331
:10462000012202210248FCF799FC10BD030800F0AA
:104630000070004070B504460D46042C02DB4FF0BC
:10464000FF3070BD04EB4400254911F8200028B16B
:1046500004EB440001EB8000407810B94FF0FF30CC
:10466000EFE774B935B9F72208214FF04020FCF785
:1046700090FD32E0F72208214FF04020FCF789FD41
:104680002BE0012C0CD12DB9EF2210211548FCF79D
:1046900080FD22E0EF2210211248FCF77AFD1CE099
:1046A000022C0CD12DB9FB2204210F48FCF771FD1F
:1046B00013E0FB2204210C48FCF76BFD0DE0032CFA
:1046C0000BD12DB9FB2204210848FCF762FD04E060
:1046D000FB2204210548FCF75CFD0020B1E7000047
:1046E000D800002000500040007000400050024000
:1046F0002DE9FE4304460F4690461E460A9D042CB3
:1047000003DA042D01DB102D03DD4FF0FF30BDE88F
:10471000FE8304EB4400A94911F8200010B94FF0C2
:10472000FF30F4E704EB4400A44901EB800040783B
:10473000012801D10020EAE7002C48D1A048FEF76B
:1047400015FBA048FEF712FB9E48FEF70FFB9D48A5
:10475000FEF70CFB9B48FEF709FB40F60F00FCF749
:10476000C3FC40F60F40FCF7BFFC41F20F00FCF722
:10477000BBFC41F20F40FCF7B7FC04214FF0402096
:10478000FCF7F8FC08214FF04020FCF7F3FC102167
:104790004FF04020FCF7EEFC20214FF04020FCF7CA
:1047A000E9FCFEF7FDFA814643463A46494686480B
:1047B000CDE90065FEF758FA8348FEF7A1FA00BF7D
:1047C00002A98148FEF784FA0028F9D1D6E0012C2D
:1047D00045D17B48401CFEF7C9FA7A48401CFEF7D9
:1047E000C5FA7848401CFEF7C1FA7648001DFEF76E
:1047F000BDFA7448001DFEF7B9FA7448FCF774FC62
:104800007348FCF771FC7348FCF76EFC7248FCF7C8
:104810006BFC20217148FCF7ADFC10216F48FCF7C0
:10482000A9FC10216E48FCF7A5FC20216C48FCF780
:10483000A1FCFEF7B5FA814643463A464946694827
:10484000CDE90065FEF710FA6648FEF759FA00BF99
:1048500002A96448FEF73CFA0028F9D18EE0022C48
:1048600045D15748801CFEF781FA5648C01CFEF718
:104870007DFA5448C01CFEF779FA5248C01CFEF776
:1048800075FA5048C01CFEF771FA5748FCF72CFC2B
:104890005648FCF729FC5648FCF726FC5548FCF71F
:1048A00023FC08215448FCF765FC04215248FCF71E
:1048B00061FC02215048FCF75DFC01214E48FCF7E9
:1048C00059FCFEF76DFA814643463A4649464B4845
:1048D000CDE90065FEF7C8F94848FEF711FA00BFB8
:1048E00002A94648FEF7F4F90028F9D146E0032C66
:1048F00044D13348401CFEF739FA3248401DFEF7D8
:1049000035FA3048401DFEF731FA2E48401DFEF7BB
:104910002DFA2C48401DFEF729FA3948FCF7E4FB34
:104920003848FCF7E1FB3848FCF7DEFB3748FCF77A
:10493000DBFB08213648FCF71DFC04213448FCF75A
:1049400019FC02213248FCF715FC01213048FCF724
:1049500011FCFEF725FA814643463A4649462D4862
:10496000CDE90065FEF780F92A48FEF7C9F900BFD6
:1049700002A92848FEF7ACF90028F9D1012004EB80
:1049800044010E4A02EB8101487004EB44001146D9
:1049900001EB800080F8098004EB440001EB80000B
:1049A000857204EB440001EB8000466004EB440098
:1049B00001EB800007720020A9E60000D80000206B
:1049C000001C00F0000800F0008000400F140100FF
:1049D0000F1001000F1004000F14040000500040DD
:1049E00000400240009000400F0C03000F0803003D
:1049F0000F0403000F0003000070004000A00040FF
:104A00000E0C05000E0805000E0405000E00050042
:104A10000050024000B000402DE9FC4704460E461D
:104A2000174698460A9D042C03DB4FF0FF30BDE883
:104A3000FC8745B12878042802DB2878102802DD9D
:104A40004FF0FF30F3E704EB4400764911F8200003
:104A500028B104EB440001EB8000407810B94FF01E
:104A6000FF30E4E702E00120FDF794FA04EB440094
:104A70006C4901EB8000C07A0128F4D0012004EBDE
:104A80004401684A02EB8101C8722EB1307804EB10
:104A9000440102EB8101087237B1387804EB44011C
:104AA000604A02EB81014872B8F1000F07D004EBB5
:104AB00044015C4A02EB8101D8F80000486035B13E
:104AC000287804EB4401574A02EB8101887234BB19
:104AD0005548FEF710F9FEF763F9814604EB4400F0
:104AE000504901EB8000807A04EB44014D4A02EB0F
:104AF00081014968CDE9001004EB4400114601EB47
:104B00008000437A04EB440001EB8000027A4946BE
:104B10004548FEF7A9F84448FEF7F2F879E0012C81
:104B200026D14248FEF7E7F8FEF73AF9814604EB52
:104B300044003C4901EB8000807A04EB4401394A8F
:104B400002EB81014968CDE9001004EB44001146F5
:104B500001EB8000437A04EB440001EB8000027A11
:104B600049463148FEF780F83048FEF7C9F850E072
:104B7000022C26D12E48FEF7BEF8FEF711F9814629
:104B800004EB4400274901EB8000807A04EB4401E8
:104B9000244A02EB81014968CDE9001004EB44008E
:104BA000114601EB8000437A04EB440001EB8000E6
:104BB000027A49461C48FEF757F81D48FEF7A0F850
:104BC00027E0032C25D11B48FEF795F8FEF7E8F8FF
:104BD000814604EB4400134901EB8000807A04EB2A
:104BE0004401104A02EB81014968CDE9001004EB51
:104BF0004400114601EB8000437A04EB440001EBD2
:104C00008000027A49460848FEF72EF80948FEF768
:104C100077F8002004EB4401024A02EB8101C872DC
:104C200000BF04E7D8000020008000400090004052
:104C300000A0004000B00040F8B504460E461546FE
:104C4000002000900027042C00DA15B94FF0FF3047
:104C5000F8BD04EB4400534911F8200028B104EBDF
:104C6000440001EB8000407810B94FF0FF30EFE7CF
:104C700002E00A20FDF78EF904EB4400494901EBFC
:104C80008000C07A0128F4D0012004EB4401454A99
:104C900002EB8101C872FBF721FB0746DCB902E099
:104CA0000120FDF777F969463F48FEF711F8002823
:104CB000F6D131463C48FEF716F802E00120FDF738
:104CC00069F93948FDF7CBFF0028F7D16946364826
:104CD000FDF7F5FF58E0012C1BD102E00120FDF7A4
:104CE00059F969463148FDF7F3FF0028F6D13146FE
:104CF0002E48FDF7F8FF02E00120FDF74BF92B48A5
:104D0000FDF7ADFF0028F7D169462848FDF7D7FF2A
:104D10003AE0022C1BD102E00120FDF73BF9694685
:104D20002348FDF7D5FF0028F6D131462048FDF78E
:104D3000DAFF02E00120FDF72DF91D48FDF78FFF96
:104D40000028F7D169461A48FDF7B9FF1CE0032C8B
:104D50001AD102E00120FDF71DF969461548FDF75B
:104D6000B7FF0028F6D131461248FDF7BCFF02E03C
:104D70000120FDF70FF90F48FDF771FF0028F7D16B
:104D800069460C48FDF79BFF3846FBF7ABFA00205D
:104D900004EB4401034A02EB8101C87200982870B9
:104DA000002055E7D800002000800040009000401F
:104DB00000A0004000B0004010B5FFF715FCFFF761
:104DC00015FCFCF78DFA10BD10B5FCF705FC0121B0
:104DD0000548FEF796F805480068401C034908603E
:104DE000FCF714FC10BD000000000340202200204E
:104DF00010B5FCF7F1FB01210548FEF782F80548E4
:104E00004068401C03494860FCF700FC10BD0000EE
:104E1000001003402022002010B5FCF7DDFB01212B
:104E20000548FEF76EF805488068401C0349886015
:104E3000FCF7ECFB10BD0000002003402022002006
:104E400010B5FCF7C9FB01210548FEF75AF80548E3
:104E5000C068401C0349C860FCF7D8FB10BD0000C7
:104E6000003003402022002010B5FCF7B5FB0121E3
:104E70000548FEF746F805480069401C03490861EB
:104E8000FCF7C4FB10BD00000040034020220020BE
:104E900010B5FCF7A1FB01210548FEF732F80548E3
:104EA0004069401C03494861FCF7B0FB10BD00009D
:104EB000005003402022002010B5FCF78DFB01219B
:104EC0000548FEF71EF805488069401C03498861C3
:104ED000FCF79CFB10BD000000000E4020220020CB
:104EE00010B5FCF779FB01210548FEF70AF80548E3
:104EF000C069401C0349C861FCF788FB10BD000075
:104F000000100E402022002070B504460D46082CEB
:104F100002DB4FF0FF3070BD34BBA948FDF726FF20
:104F20002221A848FDF7B6FFFDF73AFF4FF47A714A
:104F3000B0FBF1F000FB05F63246FF21A148FDF77A
:104F4000E6FF2320FCF792F99F491320FBF77AFD37
:104F50001320FBF70CFB01219A48FDF7D4FFFF213A
:104F60009848FDF7C7FF28E1012C27D19448401C41
:104F7000FDF7FCFE22219548FDF78CFFFDF710FFA1
:104F80004FF47A71B0FBF1F000FB05F63246FF21D9
:104F90008E48FDF7BCFF2520FCF768F98C491520E9
:104FA000FBF750FD1520FBF7E2FA01218748FDF7DA
:104FB000AAFFFF218548FDF79DFFFEE0022C27D1C7
:104FC0007F48801CFDF7D2FE22218248FDF762FF58
:104FD000FDF7E6FE4FF47A71B0FBF1F000FB05F649
:104FE0003246FF217B48FDF792FF2720FCF73EF970
:104FF00079491720FBF726FD1720FBF7B8FA0121A6
:105000007448FDF780FFFF217248FDF773FFD4E07D
:10501000032C27D16A48C01CFDF7A8FE22216F4847
:10502000FDF738FFFDF7BCFE4FF47A71B0FBF1F0ED
:1050300000FB05F63246FF216848FDF768FF332084
:10504000FCF714F966492320FBF7FCFC2320FBF74F
:105050008EFA01216148FDF756FFFF215F48FDF7F9
:1050600049FFAAE0042C27D15548001DFDF77EFE1C
:1050700022215C48FDF70EFFFDF792FE4FF47A7196
:10508000B0FBF1F000FB05F63246FF215548FDF775
:105090003EFF4F20FCF7EAF853493F20FBF7D2FCD4
:1050A0003F20FBF764FA01214E48FDF72CFFFF215A
:1050B0004C48FDF71FFF80E0052C27D14048401DDC
:1050C000FDF754FE22214948FDF7E4FEFDF768FE96
:1050D0004FF47A71B0FBF1F000FB05F63246FF2188
:1050E0004248FDF714FF5120FCF7C0F84049412029
:1050F000FBF7A8FC4120FBF73AFA01213B48FDF7FA
:1051000002FFFF213948FDF7F5FE56E0062C27D1B6
:105110002B48801DFDF72AFE22213648FDF7BAFEF6
:10512000FDF73EFE4FF47A71B0FBF1F000FB05F69F
:105130003246FF212F48FDF7EAFE7220FCF796F871
:105140002D496220FBF77EFC6220FBF710FA01215B
:105150002848FDF7D8FEFF212648FDF7CBFE2CE0BE
:10516000072C27D11648C01DFDF700FE2221234839
:10517000FDF790FEFDF714FE4FF47A71B0FBF1F0ED
:1051800000FB05F63246FF211C48FDF7C0FE7420E7
:10519000FCF76CF81A496420FBF754FC6420FBF719
:1051A000E6F901211548FDF7AEFEFF211348FDF792
:1051B000A1FE02E04FF0FF30ADE60020ABE60000BC
:1051C000000400F000000340C94D0000001003403F
:1051D000F14D000000200340194E00000030034054
:1051E000414E000000400340694E00000050034063
:1051F000914E000000000E40B94E000000100E401D
:10520000E14E000010B54FF08040FDF79BFEFDF72A
:10521000C7FD044621464FF08040FDF78CFE4FF05D
:105220008040FDF784FE10BD10B54FF07040FDF7D3
:105230009DFD2220FCF71AF84FF08040FDF782FE1A
:10524000FDF7AEFD044621464FF08040FDF773FEAA
:105250004FF08040FDF771FE4FF08040FDF767FE94
:1052600005491220FBF7EEFB1220FBF780F94FF007
:105270008040FDF754FE10BD7D52000010B5FCF7D4
:10528000ABF90C480078401C0A49087008460078C1
:105290001E2802DD0120084908700748007828B957
:1052A0004FF08040FDF740FEFFF7ACFFFCF7AEF992
:1052B00010BD000008010020090100202DE9FF4F6A
:1052C000ADF54F7D89461646DDF870830025002731
:1052D000002041904FF4807101A8FBF774F8CF983B
:1052E00060B1CF98FBF796F840B1B9F1000F05D047
:1052F000B8F1000F02D00EB1D29828B94FF0FF30AC
:105300000DF5537DBDE8F08F00240FE056F8240022
:1053100040B156F82400FBF77DF818B1D29850F848
:10532000240010B94FF0FF30EAE7641CDD98844296
:10533000ECDB012243A8CF9902F022FBCE90CE985D
:1053400010B16FF00100DBE70024FDE0ECE043AAC0
:105350004FF4807101A801F0BEFD4290429888B9D7
:1053600046994898884201D1012000E0002018B1F8
:10537000002048F82400E1E043A801F09BFD6FF015
:105380000200BDE7002700250EE0FAF7FFFF0068E6
:1053900001A9495D405C00F0010020B901A8405D11
:1053A00001A9C8557F1C6D1C01A8FBF733F8A84262
:1053B000EBD8002001A9C8559DF80400232800D18E
:1053C000B2E059F8241001A8FBF708F8B0B19DF835
:1053D00004005B2812D101A8FBF71CF8401E01A9AC
:1053E000085C5D280AD101A8FBF714F8A0F1020AB5
:1053F00059F82400FBF70EF8824500D094E087E0CE
:1054000043AA4FF4807101A801F065FD42904298D3
:1054100088B946994898884201D1012000E00020CF
:1054200018B1002048F824007CE043A801F042FDB8
:105430006FF0020064E7002700250EE0FAF7A6FFF0
:10544000006801A9495D405C00F0010020B901A895
:10545000405D01A9C8557F1C6D1C01A8FAF7DAFF51
:10546000A842EBD8002001A9C8559DF804002328C4
:1054700000D14DE056F8241001A8FAF7AFFFA8B309
:105480003D2101A8FAF7BCFF80B33D2101A8FAF73E
:10549000B7FF824600208AF8000001A8FAF7BAFF99
:1054A000834656F82400FAF7B5FF834500D02FE075
:1054B0000AF1010A5046FAF7ADFF58F82410884265
:1054C00005D943A801F0F6FC4FF0FF3018E750462D
:1054D000FAF7A0FF8346D29951F824005A46514664
:1054E000FAF758FF4198401C41901BE0FFE79DF8F8
:1054F00004005B280BD101A8FAF78CFF401E01A91C
:10550000085C5D2803D1002048F824000AE000BFB1
:1055100046994898884201D1012000E000200028E7
:105520003FF46EAF00BF09E046994898884201D128
:10553000012000E0002000283FF409AF00BF002157
:1055400043A801F0F0FC641CDD988442FFF6FEAE37
:1055500043A801F0AFFC4198D2E670B50446601C48
:1055600000F002F945B2002D02DA4FF0FF3070BDB5
:10557000A01C00F09FF845B2002D02DA4FF0FF307A
:10558000F5E7E01C00F069F845B2002D02DA4FF0B3
:10559000FF30ECE7201D00F033F845B2002D02DAB1
:1055A0004FF0FF30E3E7601D00F0B1F845B2002D89
:1055B00002DA4FF0FF30DAE7A01D00F001F945B242
:1055C000002D02DA4FF0FF30D1E70020CFE70000D6
:1055D00010B500231A4609490120FDF7B9FC04461D
:1055E000002C02DA4FF0FF3010BD902000F033F9AC
:1055F000002000F01BF90020F6E70000801A0600EA
:105600007CB504460320019000200090012301AAEC
:105610006F211846FEF734FB45B2002D02DA4FF039
:10562000FF307CBD01236A466F211846FDF7B4FEAA
:1056300045B2002D02DA4FF0FF30F2E79DF800008E
:1056400000F00F009DF80010C1F3011101EB810182
:1056500000EB410020700020E3E77CB50446022007
:10566000019000200090012301AA6F211846FEF747
:1056700007FB45B2002D02DA4FF0FF307CBD01235D
:105680006A466F211846FDF787FE45B2002D02DA03
:105690004FF0FF30F2E79DF8000000F00F009DF89A
:1056A0000010C1F3011101EB810100EB41002070FA
:1056B0000020E3E77CB50446012001900020009023
:1056C000012301AA6F211846FEF7DAFA45B2002D30
:1056D00002DA4FF0FF307CBD01236A466F21184685
:1056E000FDF75AFE45B2002D02DA4FF0FF30F2E727
:1056F0009DF8000000F00F009DF80010C1F30211AA
:1057000001EB810100EB410020700020E3E77CB554
:1057100004460420019000200090012301AA6F217B
:105720001846FEF7ADFA45B2002D02DA4FF0FF3011
:105730007CBD01236A466F211846FDF72DFE45B258
:10574000002D02DA4FF0FF30F2E79DF8000000F084
:105750000F009DF80010C1F3001101EB810100EB77
:10576000410020700020E3E77CB504460020019052
:105770000090012301AA6F211846FEF781FA45B275
:10578000002D02DA4FF0FF307CBD01236A466F2105
:105790001846FDF701FE45B2002D02DA4FF0FF304A
:1057A000F2E79DF8000000F00F009DF80010C1F333
:1057B000021101EB810100EB410020700020E3E7C2
:1057C0007CB504460520019000200090012301AA29
:1057D0006F211846FEF754FA45B2002D02DA4FF059
:1057E000FF307CBD01236A466F211846FDF7D4FDCA
:1057F00045B2002D02DA4FF0FF30F2E79DF80000CD
:1058000000F00F009DF80010090901EB810100EB89
:1058100041000549098801EBC10202EB011100EBCF
:10582000810020800020DCE70A01002038B5044612
:1058300008208DF800008DF8014002236A466F2190
:105840000120FEF71DFA45B2002D02DA4FF0FF30BD
:1058500038BD0020FCE738B5044607208DF800006D
:105860008DF8014002236A466F210120FEF708FAF5
:1058700045B2002D02DA4FF0FF3038BD0020FCE7C2
:1058800010B5012000F01CFAFF2000F020FA10BD36
:1058900070B5054601220021092000F0BEF904463A
:1058A00024B91021284600F063F90446FFF7E8FF09
:1058B0000CB1012070BD0020FCE770B505464FF625
:1058C000FF7401E0601E84B2FF2000F000FAA842DD
:1058D00001D0002CF6D10CB9FF2070BD0020FCE7F0
:1058E0007FB56846FFF7D4FF10B1002004B070BD4B
:1058F0009DF8000000F0C000402809D19DF8090083
:105900009DF8081000EB0120401C84B2A50220E0A5
:105910009DF8050000F00F009DF80A1000EBD11073
:105920009DF8091001F0030100EB4100861C9DF871
:10593000080080119DF8071000EB81009DF806100B
:1059400001F0030100EB8120441CA6F1090004FAD8
:1059500000F52846CAE700007CB50820654B002208
:10596000114600900320FEF7C3FE012000F0A8F9C5
:10597000002000F08FF9002505E0FF2000F0A7F9D6
:105980000446681C85B2642DF7DB142600BF9522FF
:105990000021084600F041F90446012C04D0301ED5
:1059A000A6F101018EB2F2D1002053490870012CFA
:1059B0004AD187224FF4D571082000F02EF9012832
:1059C00047D1002506E0FF2000F081F901A94855E4
:1059D000681C85B2042DF6DB9DF80600012879D1FC
:1059E0009DF80700AA2875D14FF6FE7600BF012268
:1059F0000021372000F011F901229107292000F041
:105A00000CF9044624B1301EA6F101018EB2EED18C
:105A1000002E5FD0012200213A2000F0FEF800287D
:105A200058D1002506E0FF2000F051F901A94855A2
:105A3000681C85B2042DF6DB9DF8040000F04000E0
:105A400018B106202C49087044E004202A49087047
:105A500040E001220021372000F0DFF80122002180
:105A6000292000F0DAF80446012C17DC0220224934
:105A700008704FF6FE7600BF01220021372000F0AB
:105A8000CCF801220021292000F0C7F80446BCB15F
:105A9000301EA6F101018EB2EED111E001201649AF
:105AA00008704FF6FE7600BF01220021104600F07C
:105AB000B4F8044624B1301EA6F101018EB2F3D130
:105AC0002EB101225102102000F0A7F810B10020E1
:105AD00009490870FFF7D4FE012000F0DBF8064802
:105AE000007808B100207CBD0CB12046FBE7AA205D
:105AF000F9E7000040420F000C0100202DE9F041C1
:105B000006460F46154619480078062800D07F0241
:105B1000012D0CD101223946112000F07EF80446F7
:105B2000FCB96902304600F023F8044619E001226E
:105B30003946122000F071F8044600BF4FF400719E
:105B4000304600F015F8044606F50076681EC0B22F
:105B5000051E01D0002CF1D0012200210C2000F004
:105B60005CF8FFF78DFE2046BDE8F0810C010020B7
:105B700070B504460D46FE20FFF79FFE08B10120D8
:105B800070BD04E0FF2000F0A2F82070641C281E05
:105B9000A5F101018DB2F5D1FF2000F098F8FF20AA
:105BA00000F095F80020EBE710B5002000F088F831
:105BB00000F09AF808B9002010BDFFF761FE01203F
:105BC000FAE72DE9F04106460D4600F08DF807464C
:105BD00017B10120BDE8F081284600F078F8FD2DCE
:105BE00019D0002404E0305D00F071F8601C84B22C
:105BF000B4F5007FF7DBFF2000F069F8FF2000F02C
:105C000066F8FF2000F063F8074607F01F0005283C
:105C100001D00220DEE70020DCE72DE9F041054657
:105C20000C4617464FF00008FFF72AFEFFF7BCFFAF
:105C300010B1FF20BDE8F08145F0400000F047F8CA
:105C4000200E00F044F8C4F3074000F040F8C4F31D
:105C5000072000F03CF8E0B200F039F8384600F0D8
:105C600036F80C2D02D1FF2000F031F84FF01F085C
:105C700000BFFF2000F02BF8064606F0800030B190
:105C8000B8F10000A8F1010101F0FF08F1D13046A0
:105C9000D0E700001CB5044614B90748019001E0A4
:105CA00006480190002001AB024601460090032007
:105CB000FEF7B2FE1CBD0000400D0300003FAB012B
:105CC00010B5044621460320FEF7B4FC10BD38B5DC
:105CD0000446002000906A4621460320FEF7ACFFF0
:105CE0009DF8000038BD000038B5002400BFFF203B
:105CF000FFF7EDFF0546FF2D01D1002038BD641CE4
:105D00006FF07F40B4FBF0F100FB114050B9082068
:105D1000074B0022114600900320FEF7E9FC01200A
:105D2000FFF7CEFF6FF070408442E0D30120E5E73B
:105D300040420F002DE9F04106460F461546204827
:105D40000078062800D07F02012D0CD101223946AF
:105D50001820FFF762FF04466CBBFE213046FFF7B8
:105D600030FF044627E016480078012809D00122B8
:105D700000213720FFF751FF012229461720FFF7A6
:105D80004CFF012239461920FFF747FF044694B91A
:105D900000BFFC213046FFF714FF044606F50076ED
:105DA000681EC0B2051E01D0002CF2D0FD210020DB
:105DB000FFF707FF0446FFF763FD2046BDE8F081CB
:105DC0000C01002010B586B000240D4805900D4848
:105DD00004900D48039040200290012002A903ABDB
:105DE00004AACDE9001005A90848FFF767FA0446A0
:105DF000012C02D1002006B010BD4FF0FF30FAE7B1
:105E0000170100201F010020402200205A960000A8
:105E100010B501220EA10F4801F088FD04460D2C9B
:105E200014D14FF400730022114609A001F0D4F9F7
:105E300004465CB9012206A1002001F077FD04466A
:105E4000012203A1034801F071FD0446204610BD64
:105E5000303A0000802200200FB4084B10B504A98E
:105E600002AA039800F01CF8044602A9002000F0E2
:105E7000B8F9204610BC5DF814FB0000E361000097
:105E800002E008C8121F08C1002AFAD17047704703
:105E9000002001E001C1121F002AFBD17047000061
:105EA0002DE9FF4F8BB088460546002606E02528E1
:105EB0000BD0DDE90D1290476D1C761C2878002868
:105EC000F5D10FB03046BDE8F08F0024A146A246C0
:105ED0000122AE4900E0044315F8013F203B02FADD
:105EE00003F00842F7D128782A2810D06FF02F024B
:105EF0002878A0F13001092915D809EB890102EBB6
:105F0000410144F0020400EB01096D1CF0E758F870
:105F1000041B5FEA010903D544F40054C9F10009E8
:105F200044F002046D1C28782E2817D115F8010FB3
:105F300044F004042A280ED06FF02F022878A0F134
:105F4000300109290AD80AEB8A0102EB410100EB72
:105F5000010A6D1CF2E758F804AB6D1C28786C2818
:105F60000FD006DC4C2817D068280DD06A2814D131
:105F700004E0742810D07A280FD10DE044F4001406
:105F80000AE044F4801401E044F44014697881424A
:105F900002D104F580146D1C6D1C2878692865D029
:105FA00006DC00288DD0632827D0642806D15DE068
:105FB0006E2808D073282AD0752877D0DDE90D1215
:105FC0009047761CE0E0C4F30250022809D0032871
:105FD0000DD0D8F8001004280DD00E6008F1040888
:105FE000D2E0D8F80010F217C1E90062F6E7D8F85D
:105FF00000100E80F2E70E70F0E718F8041B8DF821
:10600000001000208DF80100EB46012003E058F855
:1060100004BB4FF0FF3061074FF0000701D40AE0E6
:106020007F1C57450DDA8742FADB1BF80710002961
:10603000F6D106E07F1C8742FCDB1BF80710002925
:10604000F8D1DDE90D23A9EB07008146214600F0D8
:10605000B1F83044C61904E0DDE90D121BF8010B5C
:1060600090477F1EF8D22146484688E058F8040B36
:10607000C4F302514FF00A0B032900D100B20429E6
:1060800000D140B2002802DA40422D2102E0210571
:1060900005D52B218DF82410012104E006E0E1074D
:1060A00010D02021F6E708AF089113E058F8040B50
:1060B000C4F302514FF00A0B032900D180B2042926
:1060C00000D1C0B20021EEE75946FAF7AAF9303103
:1060D00007F8011D0028F7D1ADEB070000F1200BF8
:1060E000600702D524F4803401E04FF0010ADA455C
:1060F00002DDAAEB0B0000E00020824600EB0B0162
:1061000008980144A9EB01000A90E00306D4DDE9F8
:106110000D2321460A9800F04DF806444FF000097F
:1061200008E009A911F80900DDE90D12904709F10D
:106130000109761C08998945F3DBE0030CD5DDE9FC
:106140000D2321460A9800F035F8064404E0DDE905
:106150000D1230209047761CBAF10001AAF1010A15
:10616000F5DC05E0DDE90D1217F8010B9047761C10
:10617000BBF10001ABF1010BF4DC0A982146DDE92B
:106180000D2300F005F806446D1C97E60928010070
:106190002DE9F041044600251E461746880404D424
:1061A00005E039462020B0476D1C641EF9D528460D
:1061B000BDE8F0812DE9F041044600251E469046D9
:1061C000C80301D5302700E02027880404D505E066
:1061D00041463846B0476D1C641EF9D52846BDE8D7
:1061E000F0810A68531C0B60107070472DE9F04174
:1061F000044688460020E070401E60634146204609
:1062000002F078FB10B10420BDE8F08104F23620E2
:1062100002F081F9074694F83850EB2D03D0E92DB0
:1062200001D0E82D34D14AF65520874208D1082202
:106230001BA104F18A0002F0DFF908B90020E3E7AE
:1062400004F1430002F067F90646701E3040F8B9C9
:10625000B6F5007F1CDBB6F5007F19DC4520055D37
:10626000B5B1681E284098B94820005D012803D0C8
:106270004820005D02280BD104F1490002F04BF9DF
:1062800030B104F14E0002F046F908B10020BBE73E
:106290004AF65520874201D10220B5E70320B3E733
:1062A000464154333220202000000000024600E026
:1062B000521C107810B110788842F9D110787047CC
:1062C000F0B503460D461E68986A021D680A778974
:1062D000B0FBF7F400BF02CA09B90020F0BD8C4240
:1062E00000D202E0641A121DF5E700BF10682044D6
:1062F000F4E70246891ED069801E884201D800203A
:1063000070475389106B03FB0100F9E72DE9F04753
:1063100080460C4604F11A0002F0FDF810B100208E
:10632000BDE8F087207800F03F00401E00EB8001C0
:1063300001EBC0054FF00109002621E01849895DF5
:10634000081902F0E8F80746B9F1000F11D0FF2D47
:106350000BD8384601F080FE824629466D1C38F87D
:10636000110001F079FE824501D00020D8E7B9463E
:1063700005E04FF6FF70874201D00020D0E7761C81
:106380000D2EDBD3207800F0400038B1B9F1000FBA
:1063900004D038F8150008B10020C1E70120BFE79C
:1063A000F09100002DE9F04782468846DAF8004077
:1063B000B8F1000F06D1276917B1E069B84215D8C6
:1063C000012713E04146504601F0CEFF0546022D5D
:1063D00002D20120BDE8F087681C08B92846F9E719
:1063E000E069A84201D92846F4E74746606908B940
:1063F0000020EFE70026474518D17E1CE069B04237
:1064000000D802263146504601F0AEFF0546012D68
:1064100001D0681C08B92846DCE73DB12569022D8A
:1064200003D3E069A84200D92F460026E6B93E46CC
:1064300000BF761CE069B04204D80226BE4201D9F2
:106440000020C7E73146504601F08EFF054605B9EA
:1064500009E0012D01D0681C08B92846BAE7BE4200
:10646000E7D10020B6E700BF4FF0FF3231462046AB
:1064700002F05AFA8146B9F1000F08D1B8F1000FC5
:1064800005D032464146204602F04EFA8146B9F127
:10649000000F0DD12661E069801E6169814202D83A
:1064A0006069401E6061207940F00100207107E0C2
:1064B000B9F1010F02D14FF0FF3000E00120064694
:1064C000304687E72DE9F34F83B081460498006892
:1064D0000090D9F80000C768002500BF684602F0A8
:1064E000EEFB02900298401C18B9062005B0BDE8EA
:1064F000F08F0298B0F5803F05D30298020C284631
:106500006D1C27F81020029884B2202C03DB2F2C5E
:1065100001D05C2C00D111E0802C06DA214693A03A
:10652000FFF7C4FE08B10620E0E7FF2D01D30620E7
:10653000DCE728466D1C27F81040CFE700BF202C71
:1065400001DA04260CE0002602E00098401C0090CE
:10655000009800782F28F8D0009800785C28F4D0B4
:10656000009904980160012D04D1681E37F81000CD
:106570002E280BD0022D24D1681E37F810002E28AB
:106580001FD1A81E37F810002E281AD1002027F896
:10659000150080460AE0A84501D22E2100E0202106
:1065A00009F1200000F8081008F10108B8F10B0FFC
:1065B000F1D346F0200109F1200000F80810002076
:1065C00094E708E0681E37F81040202C02D02E2CEB
:1065D00000D002E06D1E002DF4D100BF002027F88E
:1065E00015000DB9062081E74FF0000A01E00AF11D
:1065F000010A37F81A002028F9D0BAF1000F03D1A8
:1066000037F81A002E2801D146F0030600E06D1E6F
:1066100025B1681E37F810002E28F8D10B22202152
:1066200009F1200002F007F84FF00008C3460820E7
:10663000019000BF50460AF1010A37F8104004B932
:1066400068E0202C03D02E2C04D1AA4502D046F0BD
:106650000306EFE70198804501D2AA4516D10198BB
:106660000B2802D146F0030654E0AA4501D046F0BB
:106670000306AA4500D94DE0AA464FF008080B20B2
:1066800001904FEA8B604FEA106BD3E7802C0EDB52
:1066900046F0020640F2B511204601F0BDFC04466A
:1066A00004F0800018B104F07F0033490C5CFF2C2B
:1066B00010DD0198401E404504D846F00306DDF881
:1066C0000480B7E72212404608F1010809F12001D1
:1066D0000A5418E024B1214628A0FFF7E7FD18B1BD
:1066E0005F2446F003060EE0412C03DB5A2C01DC4C
:1066F0004BF0020B612C06DB7A2C04DC4BF0010B17
:10670000A4F1200084B2404608F1010809F12001FB
:106710000C548FE700BF99F82000E52802D105202E
:1067200089F820000198082803D14FEA8B604FEACE
:10673000106B0BF00C000C2803D00BF003000328A7
:1067400001D146F0020606F0020048B90BF0010044
:1067500008B146F010060BF0040008B146F0080638
:106760002B2000F809600020C0E60000222A3A3CF5
:106770003E3F7C7F00000000FD9100002B2C3B3D44
:106780005B5D00002DE9FF4F85B09A4603AA012109
:10679000059800F028FB18B1012009B0BDE8F08F82
:1067A000DDF80C904FF03F08082701E07806070E4F
:1067B00037B1B9FBF7F0B0FBF8F0B0F5806FF5D862
:1067C00007B9FF274FF400720021504601F033FF54
:1067D0000AF5DF764FF0000B444669E0069850F862
:1067E0002B50642D07D801D1484603E06420B9FB43
:1067F000F0F0684305466019484501D8601901D397
:10680000A9EB040505B959E0214606F1080002F09C
:10681000C6F9294606F10C0002F0C1F9079830715B
:10682000B4FBF8F0B0FBF7F00490B4FBF8F0B0FB69
:10683000F7F107FB1100C0B20290B4FBF8F008FBBF
:106840001040401CC0B2019002987070C0210498A2
:1068500001EA900001990843B0700498F070601943
:10686000401EB0FBF8F0B0FBF7F004906019401E3A
:10687000B0FBF8F0B0FBF7F107FB1100C0B20290DB
:106880006019401EB0FBF8F108FB1100401CC0B2BB
:10689000019002987071C021049801EA900001995A
:1068A0000843B0710498F07110360BF1010B2C44C1
:1068B000BBF1040F02D20CB14C458FD300BF4AF696
:1068C00055210AF5FF7002F076F9012300225146A6
:1068D000059800F0D9FA08B101205EE700205CE7D6
:1068E000014609B1002070470020FCE7014609B1CC
:1068F000002070470020FCE72DE9F04104460E46D9
:10690000D4F800800021204600F00DFA0546EDB9CC
:10691000002700BF4046A16901F0ECFF054605B124
:1069200013E0E0690078E52802D0E069007820B93A
:10693000781C0746B04201D107E00027012120461C
:1069400000F0EBF80546002DE4D000BF042D00D187
:1069500007252846BDE8F0812DE9F0470446894621
:10696000204602F087F910B10120BDE8F0874946C2
:106970002046FFF7BEFC074667634FF40072002114
:1069800004F1380001F057FE60894FF40041B1EB8B
:10699000402F01D8084601E06089400206464FF0CA
:1069A000000800E07608B6F5007F05D9304601F012
:1069B00010FBB0F10008F5D0B6F5007F17D93246CC
:1069C0000021404601F037FE760A002500E03544FC
:1069D0006089A84207D97A1960783346414600F0A9
:1069E00053FA0028F3D0404601F0F9FA10E004F120
:1069F00038080126002500E035446089A84207D9FF
:106A00007A1960783346414600F03EFA0028F3D008
:106A10006089A84201D00120A7E70020A5E72DE961
:106A2000F0470446D4F800A00021204600F07BF98E
:106A3000064616B13046BDE8F0874FF0FF08C14664
:106A40004FF0FF30E06200BF5046A16901F052FFF5
:106A5000064606B15EE0E06905780DB9042659E006
:106A6000E069C07A00F03F07A771E52D04D007F078
:106A7000080038B10F2F05D04FF0FF084FF0FF305E
:106A8000E06240E00F2F22D12B20005D00F040009B
:106A900098BB05F0400038B1E06990F80D9005F022
:106AA000BF05A8462069E06245450CD1E069407BFE
:106AB000484508D1E169DAF80C00FFF727FC10B16E
:106AC000A8F1010000E0FF2000F0FF081BE0B8F192
:106AD000000F05D1E06902F074F8484500D119E0D3
:106AE0002B20005D00F0010040B90B2204F12001D1
:106AF000E06901F081FD08B90CE004E04FF0FF0807
:106B00004FF0FF30E0620021204600F006F8064614
:106B1000002E99D000BF30468DE72DE9F0410446A4
:106B200088462768206900F12006B6F5001F01D3CA
:106B30000020A061A06910B90420BDE8F081C6F36F
:106B40000800002845D1A069401CA061606938B9DF
:106B50003889B0EB561F3CD80020A0610420ECE738
:106B60007889401E00EA562098BB2046616901F0F2
:106B7000FBFB0546012D01D80220DEE7681C08B9A1
:106B80000120DAE7F869A8421DD8B8F1000F03D157
:106B90000020A0610420D0E720466169FFF702FCD5
:106BA00005460DB90720C8E7012D01D10220C4E731
:106BB000681C08B90120C0E729463846FFF7CCFE1B
:106BC00008B10120B9E7656129463846FFF791FB16
:106BD000A0612661C6F3080107F138000844E061AE
:106BE0000020AAE72DE9FE4F044626682B20005D11
:106BF00000F0A00010B10620BDE8FE8F4FF00009A4
:106C000001E009F10109F06830F819000028F8D115
:106C10000C2204F12001684601F000FD9DF80B00F4
:106C200000F0010028B340212B2001554FF001084E
:106C30000EE04346694604F12000F26801F02EFBA5
:106C40002046FFF7ECFE054605B104E008F1010817
:106C5000B8F1640FEDD300BFB8F1640F01D1072084
:106C6000CAE7042D01D02846C6E79DF80B102B205B
:106C700001559DF80B0000F0020030B109F10C0045
:106C80000D21B0FBF1F0401C00E001200746394621
:106C90002046FFF731FE05464DBB781E071E26D065
:106CA0002069A0EB4711204600F03DF80546F5B9F4
:106CB00004F1200001F085FF824600BF3046A16943
:106CC00001F018FE054605B110E0FAB2E16953463D
:106CD000F06801F0C5FE0120F07000212046FFF7AA
:106CE0001CFF054615B9781E071EE7D100BFC5B9C0
:106CF0003046A16901F0FEFD054695B9202200212C
:106D0000E06901F098FC0B2204F12001E06901F038
:106D100085FC2B20005D00F01800E169087301205C
:106D2000F070284668E72DE9F04104460D462668D4
:106D3000B5F5001F02D205F01F0010B10220BDE81A
:106D4000F0812561A7681FB93078032800DBF76A56
:106D500047B93089B0EB551F01D80220EFE7F06A40
:106D6000A0611CE070894FEA402811E039462046B6
:106D700001F0FAFA0746781C08B90120DFE7022F74
:106D800002D3F069B84201D80220D8E7A5EB080584
:106D90004545EBD239463046FFF7ABFAA061676153
:106DA000A06908B90220CAE7A06900EB5520A061DC
:106DB000C5F3080106F138000844E0610020BEE791
:106DC00070B5054665B9FEF7C7FD044634B101202C
:106DD000FEF760FFFF20FEF77AFF01E0002070BDA4
:106DE00000BF0120FBE72DE9F04106460F4615469E
:106DF0002EBB37B1012F1AD0022F0FD0032F1BD17A
:106E000011E00020FEF75CFFFEF76EFF08B90024DA
:106E100000E001240120FEF753FF0FE04FF4007063
:106E2000288000240AE008202880002406E0FEF7DD
:106E300057FD2860002401E0042400BF00E0012485
:106E40002046BDE8F0812DE9F04106460F46904608
:106E50001C4614B90420BDE8F0816EB9E2B2414687
:106E60003846FEF74BFE054625B1FF20FEF72FFF03
:106E70000120F0E70020EEE70420ECE7014609B925
:106E8000002070470120FCE72DE9F04105460E4641
:106E90001746984665B908F0FF0239463046FEF7B6
:106EA00049FF044614B90020BDE8F0810120FBE74A
:106EB0000420F9E738B50546284600F043FF0446AC
:106EC0003CB96946284601F020FF04460CB9002071
:106ED0002860204638BD2DE9FC4780460C46914687
:106EE00000254646641E13E06B46012201A9484670
:106EF00000F052FE0098012800D00BE09DF80470CD
:106F000000BF06F8017B6D1C0A2F00D102E000BF14
:106F1000A542E9DB00BF0020307015B14046BDE856
:106F2000FC870020FBE72DE9F04F89B004460D46B1
:106F300007A9204601F0E9FE0890089808B9607C8E
:106F40000890089818B1089809B0BDE8F08FA06AB9
:106F500000287CD0681C002843D1D4F8289059F828
:106F6000040B029002200190A76867B300BF03974B
:106F7000002004900198801C019000BF05970498A0
:106F8000401C04903946204601F0EEF90746012FD7
:106F900002D802206074D7E7781C10B90120607411
:106FA000D2E70598401C8742E8D0DDE9010188421C
:106FB00005D8049849F8040B039849F8040B07987E
:106FC000C069B842D3D80198A16A0860DDE901011F
:106FD000884203D80020C9F80000FAE01120089088
:106FE000F7E0E068A84200D2E5686561002DF4D0C2
:106FF000691E2046FFF764F9A061A1690798FFF7B1
:1070000078F98246BAF1000F02D1022060749BE742
:1070100007984089401E691E00EA51208244A08AD8
:10702000C0F308000028D8D0E0695045D5D0207CB6
:1070300000F0800080B1E26907994878012304F1EB
:107040002C01FFF721FF18B1012060747CE712E0EA
:10705000207C00F07F002074079948780123524675
:1070600004F12C01FFF7EFFE10B1012060746BE713
:10707000C4F81CA0ADE0E068A84204D2207C00F077
:10708000020000B9E568606906904FF0000BC4F893
:1070900014B0002D6AD0079840894FEA402806981E
:1070A00090B1681EB0FBF8F10698401EB0FBF8F0F6
:1070B000814209D30698401EA8F10101884360610E
:1070C00060692D1AA66912E0A6687EB900212046E3
:1070D000FFF768F90646012E02D10220607433E7FB
:1070E000701C10B9012060742EE7A660A661D6B3AB
:1070F00025E0A5EB0805606940446061207C00F054
:10710000020040B100BF31462046FFF74BF906466A
:1071100036B9002515E03146204601F025F906462E
:10712000701C10B9012060740EE7012E03D9079876
:10713000C069B04202D80220607405E7A6614545E7
:10714000D7D800BF606928446061C5F3080050B11A
:1071500031460798FFF7CDF88346BBF1000F03D106
:1071600002206074F0E601E00BEB552BE1686069EA
:10717000884205D96069E060207C40F040002074BE
:10718000A08AC0F3080020B3E069584521D0207CD4
:1071900000F0800078B1E26907994878012304F192
:1071A0002C01FFF771FE10B101206074CCE6207C49
:1071B00000F07F0020740799487801235A4604F1B3
:1071C0002C01FFF740FE10B101206074BCE6C4F84A
:1071D0001CB00898B8E600002DE9FF4F99B00F46A3
:1071E000154619A801F04EF903900398002803DA18
:1071F0000B201DB0BDE8F08FFC49039851F820002A
:1072000028B10021F94A039852F820000170039830
:10721000C0B216900020159007B9F54F1698FFF7E9
:10722000CFFD0290029800F0010008B10320E0E7D2
:10723000029800F0040008B10A20DAE77868139099
:10724000139838B913AA03211698FFF7CCFD08B19B
:1072500001201390139840B11398B0F5004F04D853
:107260001398401E1399084008B1012013904FF461
:107270000079387800F00F0018907878012804DB46
:107280007878022801DC787800E001200690B9685F
:1072900089B1B968B1F5004F0DD848464FEAE97198
:1072A00009EBD1614911BA68B2FBF1F301FB13217B
:1072B00009B9B96801E04FF400710591F868B0F1BF
:1072C000807F05D8F868411E084008B9F86800E0DA
:1072D000002007900798B0FBF9F007901C98B0FBCE
:1072E000F9F01490149808B9112082E72C462CB9B3
:1072F000149901FB09F000F06CFE04460CB9112052
:1073000077E700201190109000BF11AA0121169874
:10731000FFF769FD28B115B9204600F060FE012095
:1073200067E7189800F0080040B911983F2805D980
:107330003F201090DDE91001081A11901198802863
:1073400005D215B9204600F04AFE0E2051E700BFD5
:1073500000BF0798802801D980200790189800F076
:10736000020030B1189800F0010010B94FF0030886
:107370000CE0189800F0010028B915B9204600F07B
:107380002EFE132035E74FF0020800BF00BF00BFFC
:10739000079EB8F1030F31D1A6B911984FEA504BAF
:1073A00000200490012603E00498401C049076001D
:1073B0009049049831F8100020B1049831F8100079
:1073C0005845F1D91198B0FBF6FA082000EB8A0075
:1073D0004844401EB0FBF9F0099020200A9000209C
:1073E00008904FF6F570824502D9834882453BD913
:1073F00015B9204600F0F3FD0E20FAE6A6B9119863
:107400004FEA103B00200490012603E00498401C42
:10741000049076007949049831F8100020B104985E
:1074200031F810005845F1D91198B0FBF6FA40F642
:10743000F570824503D9042000EB4A0B07E04FF0BA
:1074400001080AEB4A00401C032101EB500B0BEB37
:107450000900401EB0FBF9F0099001200A90059840
:107460004001B0FBF9F008900A99109808440F9079
:10747000069A09990F9801FB0201089808440E909A
:1074800013990E980844401E491E20EA01010E98E7
:10749000A1EB000BB8F1030F06D10A9858440A90EB
:1074A0000F9858440F9013E00698BBFBF0F100FBD7
:1074B00011B038B1ABF1010B0A98401C0A900F983B
:1074C000401C0F900698BBFBF0F109980844099006
:1074D0000E9800EB06111098081A1199884205D9E8
:1074E00015B9204600F07BFD0E2082E611990A981E
:1074F0000A1A0699099800FB11210898081AB0FB8E
:10750000F6FAB8F1030F0FD14FF6F57082450BD89C
:10751000079818B97008079000B148E015B92046DF
:1075200000F05DFD0E2064E6B8F1020F31D14FF698
:10753000F57082451CD9079830B94020B0EB460F52
:1075400002D37000079032E0189800F0020010B1EA
:107550004FF003082BE0079820B9700007908028AF
:1075600000D824E015B9204600F039FD0E2040E691
:1075700040F6F57082450CD8079820B97000079046
:10758000802800D813E015B9204600F028FD0E2011
:107590002FE6B8F1010F09D140F6F570824505D903
:1075A00015B9204600F01BFD0E2022E600E0EFE6B4
:1075B00000BF4A460021204601F03DF80B2210A1F1
:1075C000204601F02BF8494604F10B0001F0F3FAD4
:1075D00066730A9881B204F10E0001F0ECFA069885
:1075E0002074B8F1030F11D1002010E01001002029
:1075F0009C9200008C920000F5FFFF0F7E9200002D
:10760000EBFE904D53444F53352E3000059881B218
:1076100004F1110001F0CFFA1198B0F5803F06D2C5
:10762000119881B204F1130001F0C5FA04E004F1ED
:107630002000119901F0B3FAF82060753F2104F1A0
:10764000180001F0B8FAFF2104F11A0001F0B3FAB2
:1076500004F11C00109901F0A2FAB8F1030F28D12F
:1076600000F0F2FE0146009004F1430001F097FAA9
:1076700004F12400099901F092FA022104F12C008E
:1076800001F08DFA012104F1300001F094FA062195
:1076900004F1320001F08FFA802084F840002920A4
:1076A00084F84200132294A104F1470000F0B6FFD1
:1076B00019E000F0C9FE0146009004F1270001F036
:1076C0006EFA099881B204F1160001F074FA802074
:1076D00084F82400292084F8260013228BA104F1C9
:1076E0002B0000F09BFF4AF6552104F5FF7001F0D6
:1076F00062FA01232146109A1698FFF7C5FB28B1BC
:1077000015B9204600F06BFC012072E5B8F1030FBB
:1077100033D10123109A921D21461698FFF7B4FB2E
:107720004A460021204600F086FF7D49204601F0B0
:1077300036FA7C4904F5F27001F031FAAAF1010140
:1077400004F5F47001F02BFA022104F5F67001F053
:1077500026FA4AF6552104F5FF7001F02CFA0123B0
:10776000109AD21D21461698FFF78EFB0123109A1E
:10777000521C21461698FFF787FB149800FB09F26C
:107780000021204600F057FF0F980D900020049034
:1077900048E0B8F1030F10D16FF00701204601F067
:1077A000FEF94FF0FF31201D01F0F9F96FF0704143
:1077B00004F1080001F0F3F90AE0B8F1010F01D17A
:1077C000594801E06FF007000146204601F0E7F953
:1077D0000998129000BF14991298884201D9149800
:1077E00000E0129883465B4621460D9A1698FFF7F3
:1077F0004BFB28B115B9204600F0F1FB0120F8E45D
:107800004A460021204600F016FF0D9858440D907E
:107810001298A0EB0B00129012980028DBD104986C
:10782000401C0490069904988842B2D3B8F1030F23
:1078300001D1304600E00898129000BF14991298C8
:10784000884201D9149800E0129883465B4621468D
:107850000D9A1698FFF718FB28B115B9204600F0CD
:10786000BEFB0120C5E40D9858440D901298A0EB82
:107870000B00129012980028E0D100BFB8F1030F5E
:1078800002D10C2017900DE01198B0F5803F02D383
:107890000620179006E0B8F1020F01D1042000E0A5
:1078A0000120179000BF189800F0080090B91198B7
:1078B0000B9000200C9023460BA9DDE91602FEF781
:1078C00061FF0190019828B115B9204600F087FBAF
:1078D00001988EE4002211461698FFF784FA28B129
:1078E00015B9204600F07BFB012082E415B9204643
:1078F00000F075FB00207CE44E4F204E414D4520AA
:107900002020204641543332202020004E4F204E6C
:10791000414D452020202046415420202020200099
:107920005252614172724161F8FFFF00F7B582B0B7
:1079300016460398019001A800F0A4FD0546002D0D
:1079400002DA0B2005B0F0BD0C4850F825400CB110
:1079500000202070029810B1002002990870074999
:10796000029841F825000EB90020EBE7002202A999
:1079700003A800F069FE07463846E3E7100100203F
:107980002DE9F74F90B0044616461CB9092013B0F4
:10799000BDE8F08F06F03F06324603A911A800F0BB
:1079A00053FE0546002D75D1039804904FF40070E6
:1079B00000F00FFB8346BBF1000F01D11120E6E779
:1079C0000398C0F80CB004A8119900F0D9FB054643
:1079D0002DB99DF83B0000F0800000B1062506F0AF
:1079E0001C00002857D045B1042D03D104A8FFF78F
:1079F000F9F8054646F008060AE09DF8160000F082
:107A0000110008B1072503E006F0040000B10825C5
:107A1000002D51D106F0080000284DD000F014FDD3
:107A200001900B9901F10E00019901F0B8F80B9942
:107A300001F11600019901F0B2F80B99039800F0DA
:107A40004BFD814620200B99C87200220B990398A8
:107A500001F093F80B9901F11C00002101F09FF84F
:107A600001200399C870B9F1000F25D00398D0F810
:107A700034A00022494604A801F032F80546DDB9D9
:107A80005146039800F036FF0546A9F1010003991D
:107A9000086111E07BE07DB99DF8160000F0100050
:107AA00008B1042508E006F0020028B19DF8160090
:107AB00000F0010000B107254DB906F0080008B13B
:107AC00046F040060398406B20620B986062002DE0
:107AD0005AD10B99039800F0FFFCA0600B9901F1BB
:107AE0001C0000F00CFDE0600020A0620398206004
:107AF0000398C088A080267400206074E0616061F3
:107B00004FF40072002104F12C0000F094FD06F007
:107B1000200058B3E06848B3E0686061039840898A
:107B200040020290A768D4F80C800DE03946204648
:107B300000F01AFC0746012F00D80225781C00B976
:107B400001250298A8EB000815B902988045EDD8E8
:107B5000A7615DB9C8F3080040B139460398FEF744
:107B6000C8FB8246BAF1000F01D102250CE00AEBF6
:107B70005820E061E26903994878012304F12C015F
:107B8000FFF761F900B10125584600F028FA0DB160
:107B9000002020602846FAE62DE9FF4F85B0044614
:107BA00015469A46DDF818B00020CAF8000003A96F
:107BB000204601F0AAF80490049810B9607C049063
:107BC00018B1049809B0BDE8F08F207C00F00100E6
:107BD00008B90720F6E76169E068401A019001984A
:107BE000854200D9019DA8E0A08AC0F308000028C2
:107BF00074D103984089401E616900EA5129B9F1A6
:107C0000000F1FD1606910B9A06802900CE0A06A53
:107C100028B120466169FEF753FB029004E020463C
:107C2000A16900F0A1FB02900298022802D2022072
:107C30006074C7E70298401C10B901206074C1E766
:107C40000298A061A1690398FEF753FB064616B996
:107C500002206074B6E74E444FEA5528B8F1000F91
:107C600029D009EB080003994989884203D9039870
:107C70004089A0EB090803994878434632465946A3
:107C8000FFF7E1F810B1012060749BE7207C00F061
:107C9000800068B1E069801B404509D2E169891B19
:107CA0000BEB41204FF4007204F12C0100F0B6FC04
:107CB0004FEA482737E0E069B04220D0207C00F04E
:107CC000800080B1E26903994878012304F12C0116
:107CD000FFF7DAF818B10120607473E710E0207C38
:107CE00000F07F002074039948780123324604F1A4
:107CF0002C01FFF7A8F810B10120607462E7E6617B
:107D0000A08AC0F30800C0F50077AF4200D92F4623
:107D1000A08AC0F3080204F12C0011183A46584614
:107D200000F07CFC00BFED1BDAF800003844CAF814
:107D30000000BB44606938446061002D7FF454AF9B
:107D400000203FE7F8B504466946204600F0DDFF15
:107D50000646002E44D1207C00F0400000283FD091
:107D6000207C00F0800070B1E2690099487801231E
:107D700004F12C01FFF788F808B10120F8BD207C40
:107D800000F07F00207400F05FFB0746216A009836
:107D900000F0B0FD06461EBB656AE87A40F02000A0
:107DA000E8722946A268206800F0E7FE05F11C0091
:107DB000E16800F0F4FE394605F1160000F0EFFE30
:107DC000002105F1120000F0F6FE01200099C870B4
:107DD000009800F007FF0646207C00F0BF002074EA
:107DE0003046CBE72DE9FF4F83B0044615469B464E
:107DF000049800900020CBF8000001A9204600F074
:107E000084FF0290029810B9607C029018B1029829
:107E100007B0BDE8F08F207C00F0020008B9072011
:107E2000F6E700BF606928446169884202D2606950
:107E3000C0F1FF35C3E0A08AC0F3080000287DD15F
:107E400001984089401E616900EA512ABAF1000F89
:107E500026D1606938B9A76897B900212046FEF796
:107E6000A1FA07460CE0A06A28B120466169FEF736
:107E700027FA074604E02046A169FEF793FA074671
:107E800007B99FE0012F02D102206074C0E7781C7F
:107E900010B901206074BBE7A761A06800B9A760B2
:107EA000207C00F0800078B1E269019948780123D4
:107EB00004F12C01FEF7E8FF10B101206074A7E780
:107EC000207C00F07F002074A1690198FEF711FA70
:107ED000064616B9022060749AE756444FEA5529BF
:107EE000B9F1000F2BD00AEB0900019949898842AA
:107EF00003D901984089A0EB0A09019948784B46BB
:107F000032460099FEF7C0FF10B1012060747FE790
:107F1000E069801B48450ED2E069801B009A02EBA5
:107F200040214FF4007204F12C0000F077FB207C1C
:107F300000F07F0020744FEA49282BE013E0E0694D
:107F4000B0420FD0E168606988420BD2019948784D
:107F50000123324604F12C01FEF775FF10B1012018
:107F6000607455E7E661A08AC0F30800C0F50078A8
:107F7000A84500D9A846A18AC1F3080204F12C0142
:107F800050184246009900F049FB207C40F08000E8
:107F9000207400BFA5EB0805DBF800004044CBF8D7
:107FA0000000009840440090606940446061E168CE
:107FB0006069884201D9606900E0E068E060002DF6
:107FC0007FF439AF00BF207C40F0400020740020D7
:107FD0001EE710B50446204600F0D8FA10BD10B5D3
:107FE0000446204600F032F910BD000010B50246EC
:107FF0000020084B802A01DA104609E040F2B5144F
:10800000A14205D1FF2A03DCA2F1800433F8140059
:1080100010BD0000AC92000010B5024600200D4BD0
:10802000802A01D290B213E0B2F5803F10D240F224
:10803000B514A1420CD1002001E0441CA0B280285C
:1080400003DA33F810409442F7D100F18004E0B233
:1080500010BD0000AC92000070B5B0F5803F4DD26D
:1080600081B2B1F5805F01DA254E00E0254E32463F
:1080700000BF32F8023B0BB1994200DA3CE032F823
:10808000024B2512E4B21E198E4230DD092D2CD28E
:10809000DFE805F005090F13171B1F232700CE1A71
:1080A00032F8161021E0CE1A06F001068E1BB1B28E
:1080B0001BE0A1F11006B1B217E0A1F12006B1B2A8
:1080C00013E0A1F13006B1B20FE0A1F11A06B1B28E
:1080D0000BE001F10806B1B207E0A1F15006B1B220
:1080E00003E0A1F5E356B1B200BF00BF04E0002DEC
:1080F000BFD102EB4402BCE700BF084670BD0000E0
:10810000AC9300009E9500002DE9FF4107460D4607
:1081100000213846FEF76AF80646022E06D0032EE6
:1081200000D21DB9304604B0BDE8F08100BF002484
:108130000AE007F5FB7101EB041101F1080000F002
:10814000DEF94DF82400641C042CF2D30DB1681E36
:1081500000E00020044600BF5DF8240028B15DF86F
:1081600024103846FEF742F800E0032006462DB9F9
:10817000022E03D3601C04460428EDD33046D2E718
:108180002DE9F34104462768019800782F2806D08E
:10819000019800785C2802D0B869A0600DE002E088
:1081A0000198401C0190019800782F28F8D0019880
:1081B00000785C28F4D00020A06001980078202886
:1081C00008D280212B20015500212046FEF7ABFD6F
:1081D000054637E000BF01A92046FEF773F90546C2
:1081E00005B12EE02046FEF71AFC05462B20065D61
:1081F00095B1042D0FD106F0200040B106F0040027
:1082000000B9E8E780212B200155002503E006F0A6
:10821000040000B9052514E006F0040000B110E0E8
:10822000A07900F0100008B905250AE0208AC0F303
:10823000080207F138001118384600F04DF9A06027
:10824000C9E700BF2846BDE8FC81000010B5002842
:1082500021D0114B0022001F196803E0814203D88E
:108260000A4649680029F9D152B11368841A9C4220
:1082700004D1006818441060104602E0506000E02D
:10828000186039B102680B1A934203D10B681A4483
:1082900002604968416010BD500100202DE9FF4F88
:1082A00083B0804691461E460B224046049900F05A
:1082B000B5F9052E18D9374611E039F802BB00256B
:1082C0000BE0584667F35F0007464FEA6B0B07F475
:1082D000803008B1234847406D1C102DF1D3B9F808
:1082E00000000028E9D13E46072500BF06F00F0038
:1082F00000F1300ABAF1390F03DD0AF1070000F08E
:10830000FF0A28466D1E01A901F800A03609002EBB
:10831000ECD17E20485500240AE018F80400FEF74E
:10832000DFFA20B1681EA04200D107E0641C641C83
:10833000AC4203D218F804002028EED100BF00BFE1
:10834000082D04D228466D1C01A9085C00E02020FD
:108350002146641C08F80100082CF1D307B0BDE8E1
:10836000F08F0000211001002DE9F04781460C46F6
:10837000D9F80050022C02D3E869A04202D84FF08D
:1083800001085EE04FF0FF382878012804D0022869
:108390002CD0032851D13CE0264606EB5606A86AAD
:1083A00000EB5621284600F0A5FA00B148E030461F
:1083B000761CC0F3080105F13800475CA86A00EBA1
:1083C0005621284600F096FA00B139E0C6F30801BC
:1083D00005F13800405C47EA002704F0010008B1CD
:1083E000380901E0C7F30B00804629E0A86A00EBDA
:1083F0001421284600F07EFA00B121E040F2FF117E
:1084000001EA440205F13801501800F084F8804672
:1084100016E0A86A00EBD411284600F06BFA00B110
:108420000EE040F2FF1101EA840205F13801501814
:1084300000F065F820F0704802E04FF0010800BF3E
:1084400000BF4046BDE8F0870EB56846FDF785F8E9
:10845000BDF80600A0F2BC7040069DF8051040EA89
:1084600041509DF8041040EA01409DF8031040EA95
:10847000C1209DF8021040EA41109DF80110084308
:108480000EBD000070B504464FF0FF30266831463F
:10849000324601B970BD00BF12F8013B202B01D359
:1084A0003A2BF9D13A2B11D101250E78302E08DB69
:1084B0000E78392E05DC8E1C964202D10E78A6F17C
:1084C0003005012D01DA28462260E3E7014E3078BD
:1084D00000BFDFE71601002070B505460C4604F129
:1084E0001A0000F018F806462878032805D104F190
:1084F000140000F010F846EA0046304670BD014610
:10850000C8788A7842EA00204A7842EA00200A784D
:1085100042EA00207047014648780A7842EA002083
:108520007047000088B006A90FA0F8F727FCF7F7FE
:10853000A5FEF9F717F8032000214FF480720E4BC7
:10854000CDE90132CDE90310022003460B4A009029
:108550000B48F9F711FA07AA0AA10220F9F728FB3C
:10856000F9F7BAF900BFFEE7544D344331323934DC
:108570004B43504454000000602700205C2B002037
:10858000190500005374617274000000F0B50B30DF
:10859000154D20F007010024144A0FE003688B42B8
:1085A0000BD38B4205D95E1A43184768C3E90067AD
:1085B00000E04368136002C004E0021D1068002858
:1085C000ECD12046002802D1286808B10020F0BD77
:1085D000064A07481060074A121A22F00702C0E94B
:1085E000002401202860D7E754010020500100201A
:1085F000642B0020605B0020F0B503461D460C464E
:10860000002000BF15F8017B14F801CBA7EB0C008C
:10861000561E321E01D00028F4D0F0BD30B50346FE
:108620000C463AB100BF14F8015B03F8015B551E1C
:108630002A1EF8D130BD10B5034600BF03F8011B58
:10864000541E221EFAD110BD2DE9F74F84B000212F
:10865000059801600498FFF715FF03900398002820
:1086600003DA0B2007B0BDE8F08F9D49039851F85D
:1086700020400CB90C20F5E705980460069800F03E
:10868000FE000690207878B16078FEF7F7FB074689
:1086900007F0010040B9069820B107F0040008B1C6
:1086A0000A20DFE70020DDE70020207003986070DB
:1086B0006078FEF785FB074607F0010008B103204C
:1086C000D0E7069820B107F0040008B10A20C9E7F6
:1086D00000212046FFF718FD0546042D01D1012099
:1086E000C0E7022D01D30D20BCE7D4F8349004F18B
:1086F0004300FFF710FFB0F5007F01D00D20B1E778
:1087000004F14E00FFF707FF064626B904F15C00AE
:10871000FFF7F5FE064626624820005DA070A078AF
:10872000012804D0A078022801D00D209AE7A07873
:1087300046434520005D6081608918B16089411E13
:10874000084008B10D208DE704F14900FFF7E3FE72
:108750002081207A00F00F0008B10D2082E704F19B
:108760004B00FFF7D8FE8246BAF1000F04D104F1A6
:108770005800FFF7C4FE824604F14600FFF7CBFE27
:108780008346BBF1000F01D10D206BE70BEB060018
:10879000218900EB111002900298824501D20D2030
:1087A00060E70298AAEB00006189B0FBF1F8B8F12C
:1087B000000F01D10D2055E700254A48804500D81B
:1087C00003254FF6F570804500D8022540F6F57078
:1087D000804500D801250DB90D2043E708F10200BE
:1087E000E061C4F8249009EB0B00A06202984844B1
:1087F0002063032D13D104F16200FFF78CFE08B152
:108800000D202FE7208908B10D202BE704F164002B
:10881000FFF775FEE062E0698000019014E02089B6
:1088200008B90D201EE7A06A3044E062022D02D193
:10883000E069400007E0207F00F00100E16901EB02
:10884000410100EB51000190216A019800F2FF10F4
:10885000B1EB502F01D20D2004E74FF0FF306061E3
:10886000206180202071032D2DD104F16800FFF7D5
:1088700052FE012827D109F10101204600F03AF803
:1088800008BB0020207104F23620FFF744FE4AF6B0
:108890005521884217D104F13800FFF730FE124904
:1088A000884210D104F50770FFF729FE0F4988426E
:1088B00009D104F50870FFF722FE606104F5097024
:1088C000FFF71DFE2061257009480088401C80B21A
:1088D00007490880E0800020A06100BFC2E60000D8
:1088E00010010020F5FFFF0F525261417272416189
:1088F0001401002070B504460D460026606BA842A6
:1089000010D0204600F0B6F906465EB96078012323
:108910002A4604F13801FEF796FA10B14FF0FF3500
:1089200001266563304670BD2DE9F04704460D46CB
:1089300016464FF00209022D74D3E069A84271D99E
:108940002078012804D0022849D003280DD15EE008
:108950002F4607EB5707A06A00EB57212046FFF789
:10896000C9FF8146B9F1000F00D075E038467F1C81
:10897000C0F3080104F1380001EB000805F0010024
:1089800028B1F1B298F8000061F31F1000E0304602
:1089900088F800000120E070A06A00EB5721204613
:1089A000FFF7A8FF8146B9F1000F00D054E0C7F3EC
:1089B000080104F1380001EB000805F0010010B1D6
:1089C000C6F3071006E098F8000000F0F000C6F3C8
:1089D0000321084388F800000120E0703CE0A06A11
:1089E00000EB15212046FFF785FF8146B9F1000F06
:1089F00000D031E0B1B240F2FF1202EA450304F1C7
:108A00003802981800F0D7F80120E07024E0A06A3E
:108A100000EBD5112046FFF76DFF8146B9F1000F3D
:108A200001D019E019E040F2FF1101EA850204F1DA
:108A300038015018FFF763FD66F31B00064640F24D
:108A4000FF1101EA850204F138015018314600F0A7
:108A5000A6F80120E07000BF00BF4846BDE8F087DF
:108A60002DE9F04707460C461546984684F80D80D8
:108A70000F20E07200202073002104F11A0000F0A2
:108A80009AF8681E00EB800101EBC0090020064641
:108A9000824600BF4FF6FF70864204D0484609F177
:108AA000010937F810600D4911F80A10081931460C
:108AB00000F081F80EB94FF6FF760AF10100824608
:108AC0000D28E7D34FF6FF70864202D037F8190021
:108AD00008B945F040052570BDE8F087F091000029
:108AE0002DE9F04781460E4617464FF00008D9F8A9
:108AF0000040022E02D3E069B04202D80220BDE855
:108B0000F08767B100BF4FF0FF3239462046FFF7CC
:108B10000BFF8046B8F1000F01D04046EFE700BFE1
:108B200031464846FFF720FC054605B922E0012DF5
:108B300001D10220E3E7681C08B90120DFE7002229
:108B400031462046FFF7F0FE8046B8F1000F01D015
:108B50004046D4E7E069801E6169814206D26069BF
:108B6000401C6061207940F0010020712E46E069D0
:108B7000B042D5D800BF0020C1E770B506460C460C
:108B80001546A9B204F11A0000F015F83078032850
:108B900004D1290C04F1140000F00DF870BD00F8A8
:108BA000011B090A00F8011B090A00F8011B090A48
:108BB00000F8011B704700F8011B091200F8011BA7
:108BC000704730B5014600200B2200BF431003EB75
:108BD000C01411F8015B6319D8B2531E1A1EF5D1E7
:108BE00030BD000070B50446204600F043F805464D
:108BF000002D38D1207803282ED1207901282BD1BF
:108C00004202002104F13800FFF715FD4AF6552114
:108C100004F23620FFF7CFFF144904F13800FFF7C4
:108C2000BEFF134904F50770FFF7B9FF04F508709C
:108C30006169FFF7B4FF04F509702169FFF7AFFF21
:108C4000606A401C60636078012304F13801626B44
:108C5000FEF71AF900202071607800221146FEF715
:108C6000C2F800B10125284670BD00005252614192
:108C70007272416170B504460025E078E8B1607811
:108C8000012304F13801626BFEF7FEF8A0B9002061
:108C9000E070A16A606B401A216A88420DD2A07808
:108CA00002280AD1236A616BCA186078012304F193
:108CB0003801FEF7E9F800E00125284670BD2DE9EE
:108CC000F0410646356815F8014B2046FDF708FED1
:108CD00060B115F8017B3846FDF708FE18B94FF072
:108CE000FF30BDE8F08107EB042084B24CB140F2C4
:108CF000B5112046FFF77AF9044614B94FF0FF305A
:108D0000EFE7A04635604046EBE770B504460D46F8
:108D100009268CB1206878B12068007860B1A088FD
:108D20002168C988884207D121684878FEF7A6F8EB
:108D300000F0010000B900260EB9206800E0002014
:108D40002860304670BD0000004000401000000068
:108D5000008005401000000000500040110000009D
:108D6000009005401100000000600040120000006B
:108D700000A0054012000000007000401300000039
:108D800000B0054013000000004002401400000045
:108D900000C0054014000000005002402E000000FA
:108DA00000D005402E000000006002402F000000AF
:108DB00000E005402F00000000700240300000007D
:108DC00000F005403000000000D0034046000000E5
:108DD000000006404600000000100640470000006A
:108DE0000020064048000000003006407F000000E0
:108DF0000040064080000000005006408400000053
:108E0000006006408C0000000040004010000000A0
:108E100000800540100000000050004011000000DC
:108E200000900540110000000060004012000000AA
:108E300000A0054012000000007000401300000078
:108E400000B0054013000000004002401400000084
:108E500000C0054014000000005002402E00000039
:108E600000D005402E000000006002402F000000EE
:108E700000E005402F0000000070024030000000BC
:108E800000F005403000000000D003404300000027
:108E900000000640430000000010064044000000AF
:108EA0000020064045000000003006405800000049
:108EB0000040064059000000005006405C000000E1
:108EC0000060064064000000007006406C00000076
:108ED000008006406D000000009006407F0000000A
:108EE00000400040008005400050004000900540D8
:108EF0000060004000A005400070004000B0054048
:108F00000040024000C005400050024000D0054033
:108F10000060024000E005400070024000F00540A3
:108F200000D003400000064000100640001006403C
:108F30000020064000200640003006400030064079
:108F400000400640004006400050064000500640E9
:108F50000060064000600640007006400070064059
:108F600000800640008006400090064000900640C9
:108F700000070000000600000005000000040000DB
:108F800000030000000200000001000000000000DB
:108F90000000000018ED00E01CED00E020ED00E016
:108FA00000E400E004E400E008E400E00CE400E099
:108FB00010E400E014E400E018E400E01CE400E049
:108FC00020E400E024E400E028E400E02CE400E0F9
:108FD00030E400E034E400E038E400E03CE400E0A9
:108FE00040E400E044E400E048E400E04CE400E059
:108FF00050E400E054E400E058E400E05CE400E009
:1090000060E400E064E400E068E400E06CE400E0B8
:1090100070E400E074E400E078E400E07CE400E068
:1090200080E400E084E400E088E400E000E100E0A7
:1090300004E100E008E100E00CE100E010E100E004
:1090400080E100E084E100E088E100E08CE100E004
:1090500090E100E000E200E004E200E008E200E06D
:109060000CE200E010E200E080E200E084E200E0D8
:1090700088E200E08CE200E090E200E00000010005
:1090800002000100030001000200010004000100D1
:1090900002000100030001000200010005000100C0
:1090A00002000100030001000200010004000100B1
:1090B000020001000300010002000100060001009F
:1090C0000200010003000100020001000400010091
:1090D0000200010003000100020001000500010080
:1090E0000200010003000100020001000400010071
:1090F000020001000300010002000100070001005E
:109100000200010003000100020001000400010050
:10911000020001000300010002000100050001003F
:109120000200010003000100020001000400010030
:10913000020001000300010002000100060001001E
:109140000200010003000100020001000400010010
:1091500002000100030001000200010005000100FF
:1091600002000100030001000200010004000100F0
:1091700002000100030001000200010001000000E4
:109180007856341201003F0001001800E805010084
:1091900001001000140002000A0001003F0001005D
:1091A0000100050001001800780001000400010022
:1091B0000400180008000100040001000100010083
:1091C0008000010016000100010080000100010084
:1091D000010040005800E80301001A72010010006D
:1091E00001000800E80328008002080040000A1976
:1091F00001030507090E10121416181C1E809A454B
:10920000418E418F804545454949498E8F909292C4
:109210004F994F555559999A9B9C9D9E9F41494FF7
:1092200055A5A5A6A7A8A9AAABACADAEAFB0B1B2E3
:10923000B3B4B5B6B7B8B9BABBBCBDBEBFC0C1C286
:10924000C3C4C5C6C7C8C9CACBCCCDCECFD0D1D276
:10925000D3D4D5D6D7D8D9DADBDCDDDEDFE0E1E266
:10926000E3E4E5E6E7E8E9EAEBECEDEEEFF0F1F256
:10927000F3F4F5F6F7F8F9FAFBFCFDFEFF00010048
:109280000400100040000001000200000100020084
:10929000040008001000200000000000070000008B
:1092A000000000000000000000000000C700FC00FB
:1092B000E900E200E400E000E500E700EA00EB007E
:1092C000E800EF00EE00EC00C400C500C900E600B5
:1092D000C600F400F600F200FB00F900FF00D60023
:1092E000DC00A200A300A500A7209201E100ED0090
:1092F000F300FA00F100D100AA00BA00BF00102369
:10930000AC00BD00BC00A100AB00BB0091259225C4
:10931000932502252425612562255625552563259B
:10932000512557255D255C255B2510251425342501
:109330002C251C2500253C255E255F255A25542516
:1093400069256625602550256C25672568256425D7
:10935000652559255825522553256B256A2518253D
:109360000C25882584258C2590258025B103DF00D8
:109370009303C003A303C303B500C403A603980368
:10938000A903B4031E22C603B50329226122B1003A
:109390006522642220232123F7004822B0001922ED
:1093A000B7001A227F20B200A025A00061001A0396
:1093B000E0001703F8000703FF0001007801000137
:1093C000300132010601390110014A012E017901F3
:1093D000060180014D004302810182018201840166
:1093E000840186018701870189018A018B018B0134
:1093F0008D018E018F0190019101910193019401E2
:10940000F60196019701980198013D029B019C018C
:109410009D0120029F01A001A001A201A201A401BF
:10942000A401A601A701A701A901AA01AB01AC01F2
:10943000AC01AE01AF01AF01B101B201B301B301A3
:10944000B501B501B701B801B801BA01BB01BC0152
:10945000BC01BE01F701C001C101C201C301C401C9
:10946000C501C401C701C801C701CA01CB01CA01B6
:10947000CD011001DD0101008E01DE011201F301B9
:109480000300F101F401F401F801280122021201A4
:109490003A020900652C3B023B023D02662C3F026A
:1094A00040024102410246020A015302400081018A
:1094B0008601550289018A0158028F015A029001E2
:1094C0005C025D025E025F0293016102620294012E
:1094D0006402650266026702970196016A02622CC5
:1094E0006C026D026E029C01700271029D0173029A
:1094F00074029F0176027702780279027A027B0277
:109500007C02642C7E027F02A60181028202A901F4
:109510008402850286028702AE014402B101B201D3
:1095200045028D028E028F0290029102B7017B03E9
:109530000300FD03FE03FF03AC030400860388035E
:1095400089038A03B1031103C2030200A303A30327
:10955000C4030803CC0303008C038E038F03D803DA
:109560001801F2030A00F903F303F403F503F60309
:10957000F703F703F903FA03FA0330042003500456
:109580001007600422018A043601C1040E01CF04D1
:109590000100C004D00444016105260400007D1DC3
:1095A0000100632C001E9601A01E5A01001F080630
:1095B000101F0606201F0806301F0806401F06065B
:1095C000511F0700591F521F5B1F541F5D1F561F5D
:1095D0005F1F601F0806701F0E00BA1FBB1FC81F49
:1095E000C91FCA1FCB1FDA1FDB1FF81FF91FEA1F95
:1095F000EB1FFA1FFB1F801F0806901F0806A01F05
:109600000806B01F0400B81FB91FB21FBC1FCC1F33
:109610000100C31FD01F0206E01F0206E51F010064
:10962000EC1FF31F0100FC1F4E21010032217021AD
:109630001002842101008321D0241A05302C2F042C
:10964000602C0201672C0601752C0201802C64013C
:10965000002D260841FF1A0300002F537461727415
:1096600055702E696E6900004040404040404040C7
:1096700040414141414140404040404040404040E5
:1096800040404040404040400502020202020202C7
:1096900002020202020202022020202020202020BA
:1096A00020200202020202020290909090909010FC
:1096B00010101010101010101010101010101010AA
:1096C0001010100202020202028888888888880826
:1096D000080808080808080808080808080808080A
:1096E0000808080202020240689600000C97000079
:1096F00000000020580100007404000038970000AA
:1097000058010020085A0100905E000001840A837D
:109710000178C214100853746172745570200C459E
:10972000786550617468436F6E665AFF014129087D
:08973000A94069188100000046
:0400000500000201F4
:00000001FF
